:020000040800F2
:10000000008000209D190008451700084D170008C2
:100010004F17000851170008531700080000000090
:10002000000000000000000000000000551700085C
:100030005717000800000000591700085B17000858
:10004000ED190008ED190008ED190008ED19000878
:10005000ED190008ED190008ED190008ED19000868
:10006000ED190008ED190008ED19000865170008E2
:10007000ED190008ED190008ED190008ED19000848
:10008000ED1900080000000075170008ED190008C0
:100090008D170008ED190008ED190008ED1900088A
:1000A000ED1900089D170008ED190008ED1900086A
:1000B000ED190008ED190008ED190008ED19000808
:1000C000ED190008ED190008ED190008ED190008F8
:1000D000ED190008ED190008ED190008ED190008E8
:1000E000ED190008ED190008ED190008ED190008D8
:1000F000ED190008ED190008ED19000800000000D6
:1001000000000000ED19000800000000ED190008D3
:10011000ED19000800000000ED190008ED190008B5
:10012000ED190008ED190008ED190008ED19000897
:10013000ED1900080000000000000000ED190008A3
:10014000ED190008ED190008000000000000000093
:10015000000000000000000000000000000000009F
:10016000000000000000000000000000ED19000881
:10017000ED19000800000000000000000000000071
:1001800000000000ED190008000000000000000061
:10019000000000000000000000000000000000005F
:1001A0000000000000000000ED190008ED19000833
:1001B000ED190008ED190008ED1900080000000015
:1001C00000000000ED190008000000000000000021
:0801D000ED190008ED1900080B
:1001D80010B5054C237833B9044B13B10448AFF379
:1001E80000800123237010BDB4050020000000002A
:1001F8000C92000808B5034B1BB103490348AFF341
:10020800008008BD00000000B80500200C9200081E
:1002180081F0004102E000BF83F0004330B54FEAAF
:1002280041044FEA430594EA050F08BF90EA020F1C
:100238001FBF54EA000C55EA020C7FEA645C7FEAAF
:10024800655C00F0E2804FEA5454D4EB5555B8BFD2
:100258006D420CDD2C4480EA020281EA030382EA43
:10026800000083EA010180EA020281EA0303362DD5
:1002780088BF30BD11F0004F4FEA01314FF4801CA8
:100288004CEA113102D0404261EB410113F0004FBA
:100298004FEA03334CEA133302D0524263EB430371
:1002A80094EA050F00F0A780A4F10104D5F1200E0F
:1002B8000DDB02FA0EFC22FA05F2801841F100016A
:1002C80003FA0EF2801843FA05F359410EE0A5F13E
:1002D80020050EF1200E012A03FA0EFC28BF4CF06F
:1002E800020C43FA05F3C01851EBE37101F0004525
:1002F80007D54FF0000EDCF1000C7EEB00006EEB32
:100308000101B1F5801F1BD3B1F5001F0CD34908BB
:100318005FEA30004FEA3C0C04F101044FEA445212
:1003280012F5800F80F09A80BCF1004F08BF5FEA99
:10033800500C50F1000041EB045141EA050130BD79
:100348005FEA4C0C404141EB0101013C28BFB1F58B
:10035800801FE9D291F0000F04BF01460020B1FAD6
:1003680081F308BF2033A3F10B03B3F120020CDAA9
:100378000C3208DD02F1140CC2F10C0201FA0CF087
:1003880021FA02F10CE002F11402D8BFC2F1200CEC
:1003980001FA02F120FA0CFCDCBF41EA0C019040A2
:1003A800E41AA2BF01EB0451294330BD6FEA0404EB
:1003B8001F3C1CDA0C340EDC04F11404C4F12002D6
:1003C80020FA04F001FA02F340EA030021FA04F3E8
:1003D80045EA030130BDC4F10C04C4F1200220FA3F
:1003E80002F001FA04F340EA0300294630BD21FA7D
:1003F80004F0294630BD94F0000F83F4801306BF43
:1004080081F480110134013D4EE77FEA645C18BF36
:100418007FEA655C29D094EA050F08BF90EA020FCD
:1004280005D054EA000C04BF1946104630BD91EAC5
:10043800030F1EBF0021002030BD5FEA545C05D1C8
:100448004000494128BF41F0004130BD14F5800407
:100458003CBF01F5801130BD01F0004545F0FE417B
:1004680041F470014FF0000030BD7FEA645C1ABFB0
:10047800194610467FEA655C1CBF0B46024650EAE7
:10048800013406BF52EA033591EA030F41F4002113
:1004980030BD00BF90F0000F04BF0021704730B599
:1004A8004FF4806404F132044FF000054FF000016E
:1004B80050E700BF90F0000F04BF0021704730B52F
:1004C8004FF4806404F1320410F0004548BF404204
:1004D8004FF000013EE700BF42004FEAE2014FEA59
:1004E80031014FEA02701FBF12F07F4393F07F4F34
:1004F80081F06051704732F07F4208BF704793F037
:100508007F4F04BF41F40021704730B54FF4607449
:1005180001F0004521F000411CE700BF50EA01024C
:1005280008BF704730B54FF000050AE050EA0102F5
:1005380008BF704730B511F0004502D5404261EB65
:1005480041014FF4806404F132045FEA915C3FF4A6
:10055800D8AE4FF003025FEADC0C18BF03325FEA43
:10056800DC0C18BF033202EBDC02C2F1200300FAF4
:1005780003FC20FA02F001FA03FE40EA0E0021FA19
:1005880002F11444BDE600BF70B54FF0FF0C4CF407
:10059800E06C1CEA11541DBF1CEA135594EA0C0FB9
:1005A80095EA0C0F00F0DEF82C4481EA030621EAF4
:1005B8004C5123EA4C5350EA013518BF52EA03352F
:1005C80041F4801143F4801338D0A0FB02CE4FF0E1
:1005D8000005E1FB02E506F00042E0FB03E54FF011
:1005E8000006E1FB03569CF0000F18BF4EF0010E09
:1005F800A4F1FF04B6F5007F64F5407404D25FEA05
:100608004E0E6D4146EB060642EAC62141EA5551B7
:100618004FEAC52040EA5E504FEACE2EB4F1FD0CF9
:1006280088BFBCF5E06F1ED8BEF1004F08BF5FEA77
:10063800500E50F1000041EB045170BD06F0004629
:1006480046EA010140EA020081EA0301B4EB5C04D6
:10065800C2BFD4EB0C0541EA045170BD41F48011CE
:100668004FF0000E013C00F3AB8014F1360FDEBFF3
:10067800002001F0004170BDC4F10004203C35DACF
:100688000C341BDC04F11404C4F1200500FA05F352
:1006980020FA04F001FA05F240EA020001F00042F3
:1006A80021F0004110EBD37021FA04F642EB060169
:1006B8005EEA430E08BF20EAD37070BDC4F10C0493
:1006C800C4F1200500FA04F320FA05F001FA04F257
:1006D80040EA020001F0004110EBD37041F1000143
:1006E8005EEA430E08BF20EAD37070BDC4F120054E
:1006F80000FA05F24EEA020E20FA04F301FA05F2B6
:1007080043EA020321FA04F001F0004121FA04F25D
:1007180020EA020000EBD3705EEA430E08BF20EA2D
:10072800D37070BD94F0000F0FD101F00046400067
:1007380041EB010111F4801F08BF013CF7D041EAE9
:10074800060195F0000F18BF704703F000465200ED
:1007580043EB030313F4801F08BF013DF7D043EABE
:100768000603704794EA0C0F0CEA135518BF95EA74
:100778000C0F0CD050EA410618BF52EA4306D1D1FB
:1007880081EA030101F000414FF0000070BD50EA1A
:10079800410606BF1046194652EA430619D094EAA4
:1007A8000C0F02D150EA013613D195EA0C0F05D18E
:1007B80052EA03361CBF104619460AD181EA0301E2
:1007C80001F0004141F0FE4141F470014FF000009A
:1007D80070BD41F0FE4141F4780170BD70B54FF035
:1007E800FF0C4CF4E06C1CEA11541DBF1CEA1355B5
:1007F80094EA0C0F95EA0C0F00F0A7F8A4EB050497
:1008080081EA030E52EA03354FEA013100F088808D
:100818004FEA03334FF0805545EA131343EA126356
:100828004FEA022245EA111545EA10654FEA00260B
:100838000EF000419D4208BF964244F1FD0404F5C4
:10084800407402D25B084FEA3202B61A65EB030520
:100858005B084FEA32024FF480104FF4002CB6EBDD
:10086800020E75EB030E22BFB61A754640EA0C005D
:100878005B084FEA3202B6EB020E75EB030E22BF9D
:10088800B61A754640EA5C005B084FEA3202B6EBDE
:10089800020E75EB030E22BFB61A754640EA9C009D
:1008A8005B084FEA3202B6EB020E75EB030E22BF6D
:1008B800B61A754640EADC0055EA060E18D04FEA2B
:1008C800051545EA16754FEA06164FEAC30343EACB
:1008D80052734FEAC2025FEA1C1CC0D111F4801F98
:1008E8000BD141EA00014FF000004FF0004CB6E791
:1008F80011F4801F04BF01430020B4F1FD0C88BF30
:10090800BCF5E06F3FF6AFAEB5EB030C04BFB6EB3A
:10091800020C5FEA500C50F1000041EB045170BD2D
:100928000EF0004E4EEA113114EB5C04C2BFD4EB5A
:100938000C0541EA045170BD41F480114FF0000EDE
:10094800013C90E645EA060E8DE60CEA135594EA5A
:100958000C0F08BF95EA0C0F3FF43BAF94EA0C0F5D
:100968000AD150EA01347FF434AF95EA0C0F7FF4D2
:1009780025AF104619462CE795EA0C0F06D152EA26
:1009880003353FF4FDAE1046194622E750EA41060A
:1009980018BF52EA43067FF4C5AE50EA41047FF41B
:1009A8000DAF52EA43057FF4EBAE12E74FEA41027E
:1009B80012F5001215D211D56FF47873B3EB6252A9
:1009C80012D94FEAC12343F0004343EA505311F0D0
:1009D800004F23FA02F018BF404270474FF0000062
:1009E800704750EA013005D111F0004008BF6FF0A0
:1009F800004070474FF00000704700BF4FEA4102C7
:100A0800B2F1E04324BFB3F5001CDCF1FE5C0DD964
:100A180001F0004C4FEAC0024CEA5070B2F1004FAE
:100A280040EB830008BF20F00100704711F0804FB1
:100A380021D113F13872BCBF01F00040704741F476
:100A480080114FEA5252C2F11802C2F1200C10FA7A
:100A58000CF320FA02F018BF40F001004FEAC1235E
:100A68004FEAD32303FA0CFC40EA0C0023FA02F302
:100A78004FEA4303CCE77FEA625307D150EA0133D8
:100A88001EBF4FF0FE4040F44000704701F00040A8
:100A980040F0FE4040F40000704700BF10B584B03D
:100AA80000238DF8043001A800F070F9029B9847E4
:100AB800264B83ED000A264B1A68136843F040035F
:100AC80013600A2000F0DAFF224802F0B9FE22483B
:100AD80002F0B6FE214802F0B3FE0A2000F0CEFF75
:100AE80000F064F90028FBD102221D491D4801F0DD
:100AF8005DFD1D4C0021204605F008FA0421204622
:100B080005F004FA0821204605F000FA00212046E5
:100B180005F0B8FA0421204605F0B4FA0821204669
:100B280005F0B0FA0A2000F0A9FF2268D36843F064
:100B38000103D3600A2000F0A1FF0C4B80229A61C8
:100B48000A2000F09BFF04B010BD00BFD8050020AC
:100B5800340E0020800D0020BC0D0020F80D002070
:100B6800DC050020FC0B0020980E00200010004837
:100B78001D4B1B68B3F1FF3F34D01C4A02EB8302C4
:100B880092ED007A1A49D1ED007A77EEC77AC1ED75
:100B9800007A82ED000A37EE800A81ED000A0133FF
:100BA800114A13607F2B15DD134600221A6011E0ED
:100BB8000E4A02EB830282ED000A01337F2BF7DD38
:100BC800DFED0C7A20EE270A094B83ED000A064B6D
:100BD80000221A60064B93ED000ADFED077A20EE3B
:100BE800270A70470023E9E700000020F0050020ED
:100BF800F4070020000000430000003C0000000053
:100C08002DE9F8432DED028B334CD4ED008ADFED4E
:100C1800337A78EEA78AC4ED008A314BB3F8CA005C
:100C2800B3F8A850401BFFF745FC02460B460020CE
:100C38002C49FFF7D3FD06460F462B4B588880B248
:100C4800FFF738FC22A3D3E90023FFF79DFC00221D
:100C5800264BFFF7C3FD804689462846FFF72AFC46
:100C680002460B4640464946FFF7D6FAFFF79EFE76
:100C780000B2FFF71FFC32463B46FFF785FC002217
:100C88001B4BFFF7CBFAFFF7B9FE08EE100A194E17
:100C98003060B0EE680A07F085FC28EE000AFFF71E
:100CA80067FFB0EE408A144B83ED000A94ED000A0A
:100CB80007F078FCD6ED007A9FED101AF0EE480A9E
:100CC80020EE270A00F01CF8BDEC028BBDE8F88383
:100CD8006666666666660A40F00700206F12833A09
:100CE8000075FF1F00005440DC050020000008408C
:100CF80000003E40D0050020D40500200000000080
:100D080000B585B08DED010ACDED020A8DED031A0F
:100D1800019B17480370C3F307224270C3F30742CD
:100D28008270C3F30763C370029B0371C3F3072286
:100D38004271C3F307428271C3F30763C371039B14
:100D48000372C3F307224272C3F307428272C3F3EA
:100D58000763C372002303734373802383737F2362
:100D6800C373102107F020F905B05DF804FB00BF3C
:100D7800F80700209FED010A704700BFDB0F4940CC
:100D88009FED010A704700BF0000000003781BB107
:100D9800012B04D000207047024B4360FAE7024B56
:100DA8004360F7E77D0D0008890D000838B50F4D41
:100DB8007F21284601F0C6FC0D4C7F21204601F01A
:100DC800C1FC642000F05AFE284601F009FD2A689B
:100DD800536843F020035360204601F001FD226868
:100DE800536843F020035360002038BDFC0B0020FB
:100DF800680C002010B59AB0002417941894199420
:100E08003C22214608A807F00BFB20222146684611
:100E180007F006FB3F484FF0A04303604FF4403310
:100E280043608460C46004610123436108228261D5
:100E3800047743770222026280F82440C462046384
:100E480080F83830C46380F8404000F02BFE00285A
:100E58004DD10023179317A92E4802F04DF800280A
:100E680048D12D4B08930923099301230A937F2323
:100E78000B9304230C9300230D93022210928DF8F8
:100E880044308DF845308DF84630802212924FF468
:100E9800807213928DF8503008A91E4801F01EFD8B
:100EA80058BB1E4B089340F20F13099308A9194821
:100EB80001F014FD20BB1A4B00930623019307236E
:100EC80002937F2303930423049300230593694625
:100ED800104801F0ADF8B0B9124B00930C23019300
:100EE80069460C4801F0A4F880B91AB010BD00F0AA
:100EF8008FFAAEE700F08CFAB3E700F089FAD0E792
:100F080000F086FAD7E700F083FAE5E700F080FA08
:100F1800EBE700BFFC0B00200800900C00106032CB
:100F280002003004000021C300B591B03C2200212A
:100F380001A807F075FA3548354B03604FF4403384
:100F4800436000238360C36003610122426108217A
:100F5800816103774377026280F8243080F8383063
:100F6800C36380F8403000F09DFD00283FD1294B35
:100F7800019309230293012303937F2304930422FB
:100F880005920023069309928DF828308DF82930B0
:100F98008DF82A3080220B924FF480720C928DF8D3
:100FA800343001A9194801F099FC18BB1A4B019378
:100FB80040F20F13029301A9144801F08FFCE0B925
:100FC800164B019340F21523029301A90F4801F033
:100FD80085FCA8B9124B019340F21B33029301A977
:100FE8000A4801F07BFC70B911B05DF804FB00F011
:100FF8000FFABCE700F00CFAD8E700F009FADFE7CF
:1010080000F006FAE6E700F003FAEDE7680C0020C6
:10101800000100500800900C400020198000501D6D
:1010280000018021F0B59DB0044600211791189168
:1010380019911A911B91442206A807F0F1F9236827
:10104800B3F1A04F04D05D4A934269D01DB0F0BD02
:101058004FF4004306934FF00053159306A804F08D
:101068008BF800284BD1564A136801331360012BC3
:1010780048D0544BDA6C42F00102DA64DA6C02F0C0
:1010880001020192019ADA6C42F00202DA64DB6C26
:1010980003F002030293029B05261796032718976D
:1010A8000025199517A94FF0904002F08DF90223F9
:1010B80017931897199517A9434802F085F94348DB
:1010C800434B036046608560C560802303614FF42D
:1010D800807343614FF4806383612023C361056299
:1010E80002F05AF8C8B9394B63659C6200220121A5
:1010F800122001F09DFF122001F0D2FFA6E700F0B8
:1011080087F9B0E72F4BDA6C42F40052DA64DB6CF3
:1011180003F400530093009BABE700F079F9E2E792
:101128004FF4004306934FF00053159306A804F0BC
:1011380023F8002834D1224A136801331360012BA5
:1011480031D0204BDA6C42F00402DA64DA6C02F037
:1011580004020492049ADA6C42F00102DA64DB6C4D
:1011680003F001030593059B07231793032518959F
:101178000024199417A9174802F026F94023179359
:101188001895199417A94FF0904002F01DF92246BE
:101198000121122001F04CFF122001F081FF55E7D8
:1011A80000F036F9C7E7074BDA6C42F40052DA640C
:1011B800DB6C03F400530393039BC2E70001005068
:1011C800F80B00200010024000040048D40C002056
:1011D800080002400008004800B583B00E4B9A6C26
:1011E80042F004029A649A6C02F004020092009A97
:1011F8009A6C42F001029A649B6C03F0010301931C
:10120800019B002202210B2001F012FF0B2001F0AC
:1012180047FF03B05DF804FB00100240F0B58DB045
:1012280000240794089409940A940B94394BDA6CB7
:1012380042F02002DA64DA6C02F020020192019A8C
:10124800DA6C42F00402DA64DA6C02F00402029208
:10125800029ADA6C42F00102DA64DA6C02F00102F6
:101268000392039ADA6C42F00202DA64DA6C02F052
:1012780002020492049ADA6C42F01002DA64DA6C20
:1012880002F010020592059ADA6C42F00802DA645C
:10129800DB6C03F008030693069B1F4D2246802152
:1012A800284602F07BF91D4F22460421384602F0F9
:1012B80075F9802307930126089609940A9407A9CB
:1012C800284602F081F84FF4804307930894099464
:1012D80007A9284602F078F84FF4004307930894CA
:1012E800099607A9284602F06FF84FF48063079320
:1012F8000894099407A90A4802F066F8042307939A
:10130800089609940A9407A9384602F05DF80DB0CA
:10131800F0BD00BF0010024000100048000C00485B
:101328000004004808B51548154B036003F1015344
:1013380003F57E2303F28C7343600023836001224C
:10134800C260036143618361C361036202F02BF9E8
:1013580050B90021094802F084F940B90021074832
:1013680002F0ADF930B908BD00F052F8F1E700F02D
:101378004FF8F3E700F04CF8F5E700BF340D002014
:101388000078004010B598B00446002113911491DC
:10139800159116911791442202A807F041F8226886
:1013A800184B9A4201D018B010BD4FF480730293C5
:1013B80002A803F0E1FE08BB134CE36C43F00403FE
:1013C800E364E36C03F004030093009B4FF4407361
:1013D800139312231493002315931693082317933A
:1013E80013A90A4801F0F0FFA36D43F08043A365F9
:1013F800A36D03F080430193019BD4E700F008F844
:10140800DAE700BF007800400010024000080048FA
:1014180072B6FEE700B595B03822002106A806F09E
:10142800FFFF00200190029003900490059003F0C4
:101438001BFA212306934FF48033079301230C935F
:1014480002230D9303220E920F931C2210921193E4
:101458001293139306A803F0C1FA90B90F230193CE
:1014680003230293002303930493059304210DEBB4
:10147800010003F06BFD30B903F064FE15B05DF8B0
:1014880004FBFFF7C5FFFFF7C3FF08B500F0D4FA68
:10149800FFF7C0FFFFF7C2FEFFF79EFE00F0D6F988
:1014A800FFF7A8FCFFF73EFF00F010F800F026F861
:1014B80000F03CF8FFF738FD06F024FD00F0BCF81A
:1014C800FFF7ECFAFFF79CFBFCE7000008B50948BA
:1014D800094B0360002343608360C36003610375A5
:1014E8008361C36202F018F900B908BDFFF790FFE5
:1014F800FBE700BF800D00200003014008B5094844
:10150800094B03600023436083602022C2600361AB
:1015180003758361C36202F0FFF800B908BDFFF7E5
:1015280077FFFBE7BC0D00200403014008B509481C
:10153800094B0360002343608360C3600361037544
:101548008361C36202F0E8F800B908BDFFF760FFE5
:10155800FBE700BFF80D00200803014010B58AB072
:1015680000230593069307930893099303682C4A6D
:10157800934207D02B4A934218D02B4A93423BD030
:101588000AB010BD294BDA6C42F00102DA64DB6C58
:1015980003F001030193019B0E2305930323069394
:1015A80005A94FF0904001F00FFFE9E71F4BDA6CF7
:1015B80042F00102DA64DA6C02F001020292029A45
:1015C800DA6C42F00402DA64DB6C03F00403039380
:1015D800039BC02305930324069405A94FF090406C
:1015E80001F0F2FE2023059306940023079305A932
:1015F8000F4801F0E9FEC3E70C4BDA6C42F0020237
:10160800DA64DB6C03F002030493049B072305935D
:101618000323069305A9074801F0D6FEB0E700BFEB
:101628000003014004030140080301400010024088
:10163800000800480004004808B51148114B036031
:101648004FF482734360002383604FF47062C2607A
:1016580002220261012242614FF400728261182263
:10166800C2610362436283620722C2620363436307
:1016780003F0F4FE00B908BDFFF7CAFEFBE700BFA0
:10168800340E002000300140F0B589B000230393E8
:1016980004930593069307930268184B9A4201D066
:1016A80009B0F0BD03F560431A6E42F480521A6621
:1016B8001A6E02F480520192019ADA6C42F0020228
:1016C800DA64DB6C03F002030293029B2823039382
:1016D800022404940327069705260796084D03A9B4
:1016E800284601F071FE102303930494059406978D
:1016F800079603A9284601F067FED1E700300140AC
:101708000004004800B583B00B4B1A6E42F001028A
:101718001A661A6E02F001020092009A9A6D42F05F
:1017280080529A659B6D03F080530193019B03F0EF
:1017380021F903B05DF804FB0010024008B503F07E
:101748000BFDFEE7FEE7FEE7FEE7FEE770477047A2
:10175800704708B500F080F908BD000008B50248D8
:1017680001F0D0FD08BD00BFD40C002008B5034827
:1017780000F0C2FA024800F0BFFA08BDFC0B0020D6
:10178800680C002008B5024802F02BFE08BD00BF17
:10179800BC1B002008B5024804F051F808BD00BF82
:1017A800980E0020034AD2F8883043F47003C2F838
:1017B8008830704700ED00E002680E4B9A4200D076
:1017C800704700B583B003F564431A6E42F40062B3
:1017D8001A661B6E03F400630193019B00220F211C
:1017E800192001F025FC192001F05AFC03B05DF81E
:1017F80004FB00BF002C014000B587B00023019313
:10180800029303930493059302680E4B9A4202D005
:1018180007B05DF804FB03F56443DA6C42F010028C
:10182800DA64DB6C03F010030093009B4FF47C53E5
:10183800019302230293059301A9034801F0C4FD13
:10184800E6E700BF002C01400010004810B59CB02E
:101858000024189419941A941B94159416941794A8
:101868000E940F9410941194129413941494342297
:10187800214601A806F0D4FD4448454B0360446066
:101888002023836040F6AC53C360046144618461E3
:1018980004F040F900285DD14FF48053189318A93B
:1018A8003A4804F087FA002857D1384804F062F91A
:1018B800002855D17023159300231693179315A963
:1018C800324804F059FC00284DD160230E930022C1
:1018D8000F92109211921292139214920EA92B4801
:1018E80004F0BEF9002841D104220EA9274804F0CB
:1018F800B7F900283DD108220EA9244804F0B0F910
:10190800002839D170230E9340F67A530F930C2296
:101918000EA91E4804F0A4F9002830D10023019331
:1019280002930393049305934FF40052069207938E
:10193800089309934FF000720A920B930C930D933E
:1019480001A9124804F062FCE0B91048FFF754FFFF
:101958001CB010BDFFF75CFD9EE7FFF759FDA4E73B
:10196800FFF756FDA6E7FFF753FDAEE7FFF750FD7B
:10197800BAE7FFF74DFDBEE7FFF74AFDC2E7FFF7FD
:1019880047FDCBE7FFF744FDDFE700BF980E0020D7
:10199800002C01400D4885460D480E490E4A00238B
:1019A80002E0D458C4500433C4188C42F9D30B4A0B
:1019B8000B4C002301E013600432A242FBD3FFF773
:1019C800F1FE06F009FDFFF760FDFEE7008000204C
:1019D80000000020B40500205C960008B405002033
:1019E800D4200020FEE70000104B1B680BB9012033
:1019F800704710B504464FF47A70B0FBF3F30C4A05
:101A08001068B0FBF3F001F059FB68B90F2C01D94D
:101A180001200AE0002221464FF0FF3001F008FBC8
:101A2800044B1C60002000E0012010BD08000020CD
:101A3800040000200C00002010B5032001F0E6FA95
:101A48000F20FFF7D1FF10B10124204610BD044636
:101A5800FFF758FEF9E70000034A136803490968CD
:101A68000B441360704700BFE40E002008000020FC
:101A7800014B1868704700BFE40E002038B50446D3
:101A8800FFF7F6FF0546B4F1FF3F02D0044B1B6891
:101A98001C44FFF7EDFF401BA042FAD338BD00BF3E
:101AA8000800002030B583B000230193002800F01F
:101AB8000D810446C36D13B323689A6812F0005F62
:101AC80005D09A6822F0204222F03F029A602268EC
:101AD800936813F0805F1FD1936823F0104323F0BD
:101AE8003F0343F080539360794B1B689B09794A05
:101AF800A2FB03239B0901335B00019309E0FFF775
:101B080091FA0023236684F85830D5E7019B013BFE
:101B18000193019B002BF9D12268936813F0805F31
:101B280040F09C80E36D43F01003E365236E43F0BF
:101B3800010323660120936813F0040300D00123F6
:101B4800E16D11F0100F40F0BA80002B40F0B78023
:101B5800E36D23F4817343F00203E365936813F0A4
:101B6800010F15D14FF0A0439B6813F0010300D07B
:101B78000123594A926812F0010200D0012213434E
:101B880006D1636855498A6822F47C1213438B6036
:101B9800627FE36B43EA4233E2681343A26813436C
:101BA80094F8242043EA0243012A59D0E26A22B178
:101BB80002F47872216B0A4313432168CD68484ABE
:101BC8002A401343CB602268136923F04063616B9A
:101BD8000B43136121688B6813F0040300D00123C1
:101BE8008A6812F0080200D0012243BB3ABB227F68
:101BF80094F838305B0043EA8232CB6823F48043A0
:101C080023F002031343CB60236973B3226813697B
:101C180043F4803313612268D2F8C03023F47F5331
:101C280023F03F0321690B43C2F8C03094F84030D9
:101C3800012B29D02268136923F00103136163691A
:101C4800012B33D02268136B23F00F031363E36D6A
:101C580023F0030343F00103E36535E000206AE75E
:101C6800A26A013A43EA4243A0E72268136923F4CF
:101C7800803313612268D2F8C03023F47F5323F0F5
:101C88003F03C2F8C030D1E721680B6923F4FF6332
:101C980023F00403626CA56C2A43E56C2A43256D86
:101CA8002A43134343F001030B61C8E721680B6B18
:101CB80023F00F03226A013A13430B63C7E7E36D6E
:101CC80043F01003E365012003B030BD0120FBE7BA
:101CD80004000020632D3E05000100500003005061
:101CE8000740F0FF7047704708B5806AFFF7FBFFB1
:101CF80008BD704770470000F8B5044603681F68C0
:101D08005D68984B9E6806F01F0617F0020F10D00A
:101D180015F0020F0DD0C36D13F0100F03D1C36D72
:101D280043F40063C365204600F0D6FD2368022211
:101D38001A6017F0040F02D015F0040F05D117F040
:101D4800080F4AD015F0080F47D0E36D13F0100FB5
:101D580003D1E36D43F40073E3652368DA6812F492
:101D6800406F34D1804A934209D01A46934209D031
:101D780046B1052E06D0092E04D0D26803E04FF0F4
:101D8800A042F3E7DA6812F4005F20D11A6812F073
:101D9800080F1CD09A6812F0040F10D15A6822F06C
:101DA8000C025A60E36D23F48073E365E36D13F46A
:101DB800805F0CD1E36D43F00103E36507E0E36D59
:101DC80043F01003E365236E43F0010323662046C6
:101DD800FFF788FF23680C221A6017F0200F02D043
:101DE80015F0200F05D117F0400F5CD015F0400F0B
:101DF80059D0E36D13F0100F03D1E36D43F4005392
:101E0800E3652368DA6C12F4C07F12D10121DA6825
:101E180012F4406F0FD10120534A93420DD01A4655
:101E280093420DD066B1062E0AD0072E08D0D2688C
:101E380007E00021EBE70020EEE74FF0A042EFE7D4
:101E4800DA6851B312F0007F03D030B312F4005FA8
:101E580023D1196811F0400F1FD012F4001F1CD1B4
:101E68009A6812F0080F10D15A6822F060025A607E
:101E7800E36D23F48053E365E36D13F4807F0CD1A5
:101E8800E36D43F00103E36507E0E36D43F01003FE
:101E9800E365236E43F001032366204600F018FD36
:101EA800236860221A6017F0800F02D015F0800FA7
:101EB8002FD117F4807F02D015F4807F34D117F426
:101EC800007F02D015F4007F3AD117F0100F19D017
:101ED80015F0100F16D0E36B33B1002E3CD0214B18
:101EE8009B6813F4604F0AD0E36D43F48063E365A5
:101EF800236E43F0020323662046FFF7FBFE2368A8
:101F080010221A6017F4806F02D015F4806F2DD15B
:101F1800F8BDE36D43F48033E3652046FFF7E9FE3F
:101F2800236880221A60C4E7E36D43F40033E36555
:101F3800204600F0CFFC23684FF480721A60BEE799
:101F4800E36D43F48023E365204600F0C4FC236876
:101F58004FF400721A60B8E72368DB6813F0010FCA
:101F6800CDD0C1E70003005000010050E36D43F4F9
:101F78008043E365236E43F00803236623684FF428
:101F880080621A60204600F0A4FCC1E708B5034649
:101F9800806AC26D12F0500F30D1C36D43F40073E4
:101FA800C36503681A6812F0080F14D0DA6812F4CF
:101FB800406F20D1DB6813F4005F1CD1C36D23F49C
:101FC8008073C365C36D13F4805F14D1C36D43F090
:101FD8000103C3650FE0DB6813F0020F0BD1C36D7B
:101FE80023F48073C365C36D13F4805F03D1C36D9D
:101FF80043F00103C365FFF775FE08BDC26D12F01B
:10200800100F04D1426D526B18469047F5E7FFF761
:1020180071FEF2E708B5806AC36D43F04003C365FB
:10202800036E43F004030366FFF764FE08BD000077
:10203800F0B583B00022019290F85820012A00F0F0
:102048005E820346012280F858200568A86810F0CF
:10205800040F09D0DA6D42F02002DA65012000226F
:1020680083F8582003B0F0BD4C683035220A92003E
:1020780002F00C02A85804F01F0E1F2404FA0EF4F4
:1020880020EA04000C68C4F3846C0CFA0EFC40EAE5
:102098000C00A8501868826812F0040200D00122CF
:1020A800846814F0080400D00124002A4FD1002CC1
:1020B8004DD18D68B5F1004F7CD00F6814307A0E81
:1020C800920002F004028658C7F3045E4FF0070C32
:1020D8000CFA0EFC26EA0C0C05FA0EF54CEA05057E
:1020E80085501868426922F0004242614D691868BB
:1020F800C268C2F3C102520005FA02F20E69042E48
:1021080070D0603050F82670A94D3D400F6807F038
:10211800F8473A43154345F0004540F826501A68F9
:102128000E698869603252F8265025F08075284378
:1021380042F826001A680D69087F01284FD06032DE
:1021480052F8250020F00070044342F825401A6830
:10215800906810F0010F12D10868CD68954CA5421F
:1021680000F0A780D2F8B040C0F3120024EA0000C3
:10217800C2F8B000C8688F4A904200F0A2800A688E
:102188008D490A4200F0B3818C49896801F0E070FA
:102198008B4CA24200F062818A4CA24200F05E8120
:1021A800894CA24200F08081884CA24200F08E81C6
:1021B800002054E70D6814306A0E920002F0040201
:1021C8008658C5F30455072707FA05F526EA0505D5
:1021D80085501868426942F00042426186E74FF034
:1021E8000074ACE7026E046EC4F384640A68C2F338
:1021F80012057DBBC2F38462944233D01C68626EC0
:10220800606EC0F384600A68C2F312057DBBC2F336
:102218008462904233D01C68A26EA06EC0F38460C2
:102228000A68C2F312057DBBC2F38462904233D0C0
:102238001C68E26EE06EC0F384600A68C2F312059F
:102248007DBBC2F38462904281D1E26E22F00042EB
:10225800E2667CE792FAA2F212B1B2FA82F2CBE716
:102268002022C9E7026E22F000420266C6E792FA0F
:10227800A2F212B1B2FA82F2CBE72022C9E7626E6B
:1022880022F000426266C6E792FAA2F212B1B2FAEE
:1022980082F2CBE72022C9E7A26E22F00042A266B2
:1022A800C6E792FAA2F212B1B2FA82F2CBE7202282
:1022B800C9E7D2F8B040C0F312002043C2F8B0001A
:1022C80058E71C680A68C2F31205002D38D1900E31
:1022D800013000F01F0009288CBF002001200028D1
:1022E80076D0002D3BD1900E0130800600F0F840EA
:1022F800002D40D1960E013606F01F070126BE407C
:102308003043002D45D1920E013202F01F0202EB3C
:10231800420212050243886804F11406550EAD0006
:1023280005F004057459C2F304524FF0070C0CFA77
:1023380002FC24EA0C0C90404CEA000070511EE7A5
:1023480092FAA2F048B1B0FA80F0013000F01F0014
:1023580009288CBF00200120C1E72020F5E792FA68
:10236800A2F030B1B0FA80F00130800600F0F840F9
:10237800BEE72020F8E792FAA2F646B1B6FA86F64A
:10238800013606F01F06012707FA06F6B8E72026E9
:10239800F6E792FAA2F242B1B2FA82F2013202F000
:1023A8001F0202EB42021205B4E72022F6E700BF43
:1023B80000F0FF0300007F40000008800003005089
:1023C800000021C31000C090000052C7000084CB59
:1023D800CDB9900E0130800600F0F840FDB9960E98
:1023E800013606F01F070126BE4030432DBB920E72
:1023F800013202F01F0202EB42021E3A120542F0BD
:102408000072024387E792FAA2F030B1B0FA80F086
:102418000130800600F0F840E0E72020F8E792FA63
:10242800A2F646B1B6FA86F6013606F01F0601276F
:1024380007FA06F6D9E72026F6E792FAA2F25AB189
:10244800B2FA82F2013202F01F0202EB42021E3A95
:10245800120542F00072D4E72022F3E711F4000FCE
:102468007FF49EAE1A68B2F1A04F01D00020F6E5C5
:1024780040F4000023498A6822F0E0721043886023
:10248800214A126892092149A1FB021292090132DC
:1024980002EB420292000192019A1AB1019A013AA2
:1024A8000192F9E70020DAE511F0807F7FF47CAE35
:1024B8001968174A91421CD040F0807011498A6807
:1024C80022F0E072104388600020C8E511F4800F04
:1024D80011D119680E4A91420FD040F48002094880
:1024E800816821F0E0710A4382600020B7E500208E
:1024F800B5E50020B3E50020B1E50020AFE50220F6
:10250800B0E500BF0003005004000020632D3E0525
:102518000001005038B503689A6812F0010F40D1E5
:1025280004469968204A114209D0C36D43F010034C
:10253800C365036E43F001030366012032E09A6825
:1025480022F0004222F03F0242F001029A60FFF7B7
:102558008FFA054623681A6812F0010F1FD19A688E
:1025680012F0010F07D19A6822F0004222F03F02D0
:1025780042F001029A60FFF77BFA431B022BE9D96C
:1025880023681B6813F0010FE4D1E36D43F01003D7
:10259800E365236E43F001032366012002E0002077
:1025A80000E0002038BD00BF3F000080F8B50446B9
:1025B8003A4B9D680068806810F0040F69D10E4698
:1025C800174605F01F0594F85830012B63D00123F6
:1025D80084F8583045B1052D06D0092D04D00023C4
:1025E80084F85830012055E02046FFF793FF002873
:1025F8004BD1E36D23F4706323F0010343F480733C
:10260800E3652368264A934239D01A46934200D09C
:102618001DB9E36D23F48013E365E36D13F4805F64
:1026280030D0236E23F006032366636D1D4ADA62F9
:10263800636D1D4A1A63636D1C4A5A6323681C2222
:102648001A60002384F858302268536843F0100356
:1026580053602268D36843F00103D36021683B4686
:1026680032464031606D00F003FE2268936823F023
:10267800004323F03F0343F0040393600AE04FF064
:10268800A042C3E700232366CFE7002384F858302D
:1026980000E00220F8BD0220FCE700BF0003005064
:1026A80000010050951F0008F11C00081D200008BB
:1026B80038B504460268936813F0020300D001237A
:1026C800916811F0010F39D0002B39D1936803F0CC
:1026D8000D03012B09D0E36D43F01003E365236E6E
:1026E80043F001032366012029E0936823F00043A7
:1026F80023F03F0343F002039360236803221A6028
:10270800FFF7B6F9054623689B6813F0010F13D04D
:10271800FFF7AEF9401B0228F5D923689B6813F030
:10272800010FF0D0E36D43F01003E365236E43F02F
:1027380001032366012002E0002000E0002038BDEC
:102748000020FCE730B583B00023019390F858309F
:10275800012B41D004460D46012380F85830FFF77D
:10276800A7FF80BBE36D23F4885323F0020343F0F3
:102778000203E3652268936823F0404323F03F0394
:1027880005F080452B4343F00043936023689B6822
:10279800002B06DBE36D23F0030343F00103E3653D
:1027A80015E0019B01330193019A0C4B9A42EDD934
:1027B800E36D23F0120343F01003E365002384F86C
:1027C8005830012006E0E36D43F01003E365002371
:1027D80084F8583003B030BD0220FBE701DE040066
:1027E80038B5394B9D6803689A6812F0080F67D1AD
:1027F800044605F01F05DA68DB6C13F4C07F01D1CD
:10280800002A3DDA94F85830012B5BD0012384F874
:1028180058302046FFF77EFE00284DD1E36D13F4B3
:10282800807F33D0236E23F008032366E36D23F4FF
:10283800405323F0010343F48053E3652368234A9C
:10284800934226D01A46934200D01DB9E26D22F475
:102858008012E26560221A60002384F858302368E9
:102868001A4A934218D01A46934218D0BDB1062D81
:1028780015D0072D13D0E36D43F48013E36520E0F2
:10288800C36D43F02003C36501201AE000232366CB
:10289800CCE74FF0A042D6E74FF0A042E4E7DA6871
:1028A80012F0007F0DD19A6822F0004222F03F0218
:1028B80042F008029A6004E0002384F8583000E0EF
:1028C800022038BD0220FCE7000300500001005040
:1028D800704770477047704770470000F0B583B085
:1028E800034600220192406993F85820012A00F01B
:1028F800F882012283F85820A8B10A6A012A12D066
:10290800986E002840F0CD809A6600225A668C6A3C
:10291800002C00F0C3800A6A013A04F07C042243C8
:10292800CC6A1443BEE04A68092A00F097801A6806
:10293800906810F0080F10D191F82500002840F099
:10294800D080D06820F4401091F8265091F82440A7
:10295800240544EA45542043D0601C68A26812F05C
:10296800040200D00122A56815F0080500D0012551
:10297800002A40F06181002D40F092818A6A1AB1E4
:10298800CA6A002A40F0BC8091F82520012A00F08C
:10299800B180E26822F00072E260002091F83020F5
:1029A800012A00F0BC801C68226922F00202226120
:1029B8008C68B4F1004F00F0BE801A680F6802F10D
:1029C800140C7A0E920002F004025CF80260C7F35D
:1029D80004574FF0070E0EFA07FE26EA0E06BC4013
:1029E80034434CF802401C68626922F0004262617C
:1029F8004C691E68F268C2F3C102520004FA02F27E
:102A0800D1F810C0BCF1040F00F0AF80603656F862
:102A18002C40A84F27400C6804F0F8442243174381
:102A280047F0004746F82C701A680F698C696032C5
:102A380052F8276026F08076344342F827401A6817
:102A48000E690C7F012C00F08D80603252F8264010
:102A580024F00074254342F82650EEE08C6ABCB19D
:102A68000868820E520202F4785204F07C04224371
:102A7800C86A02431C68E06C20F07B4020F46F00B9
:102A880020F43F4020F0FF001043E0645A664EE710
:102A98000A68920E520202F47852EBE70A6A541E50
:102AA80000E000240868C0F384604A6802F01F024E
:102AB80000FA02F22243986E013898665C6E22434F
:102AC8005A6600287FF433AF1C68E06C20F07B4026
:102AD80020F46F0020F43F4020F0FF000243E2643E
:102AE80025E7D06820F4401091F8264040EA445089
:102AF800D06032E7E26842F00072E26000204DE701
:102B080091F82500012805D0E26822F00072E26001
:102B1800002043E7DA6D42F02002DA653EE71E68DE
:102B2800326922F4FF724C6B8F6B3C43224342F0B4
:102B3800020232613CE71C680E681434720E92007F
:102B480002F00402A758C6F304564FF0070C0CFA1B
:102B580006F627EA0606A6501C68626942F000429B
:102B6800626145E74FF000756FE7326E346EC4F36B
:102B780084640A68C2F312057DBBC2F3846294427E
:102B880033D01D686A6E6C6EC4F384640A68C2F33D
:102B980012067EBBC2F38462944233D01D68AA6ECB
:102BA800AC6EC4F384640A68C2F312067EBBC2F337
:102BB8008462944233D01D68EA6EEC6EC4F3846478
:102BC8000A68C2F312067EBBC2F38462944234D10F
:102BD800EA6E22F00042EA662FE092FAA2F212B1FF
:102BE800B2FA82F2CBE72022C9E7326E22F0004225
:102BF8003266C6E792FAA2F212B1B2FA82F2CBE7D3
:102C08002022C9E76A6E22F000426A66C6E792FA95
:102C1800A2F212B1B2FA82F2CBE72022C9E7AA6E79
:102C280022F00042AA66C6E792FAA2F212B1B2FAFC
:102C380082F2CBE72022C9E700201A68946814F0D2
:102C4800010F10D10C68CE681B4DAE422AD0D2F8C5
:102C5800B050C4F3120425EA0404C2F8B040CC68AA
:102C6800154A944236D00A6814490A4213D01449C6
:102C7800896801F0E074134DAA4200F0E980124D12
:102C8800AA4200F0E580114DAA4200F00681104DDD
:102C9800AA4200F01481002283F8582003B0F0BD46
:102CA8000020CAE7D2F8B050C4F312042C43C2F88B
:102CB800B040D4E700F0FF0300007F400000088028
:102CC80000030050000021C31000C090000052C74C
:102CD800000084CB1D680A68C2F31206002E37D1A3
:102CE800940E013404F01F04092C8CBF0024012425
:102CF800002C65D0002E3AD1940E0134A40604F0BD
:102D0800F844002E3FD1970E013707F01F0C01271A
:102D180007FA0CF73C43002E44D1920E013202F020
:102D28001F0202EB4202120522438C681435560E2C
:102D3800B60006F00406AF59C2F304524FF0070C70
:102D48000CFA02FC27EA0C0794403C43AC518AE792
:102D580092FAA2F44CB1B4FA84F4013404F01F04DA
:102D6800092C8CBF00240124C2E72024F5E792FA3D
:102D7800A2F434B1B4FA84F40134A40604F0F8449B
:102D8800BFE72024F8E792FAA2F74FB1B7FA87F71E
:102D9800013707F01F074FF0010C0CFA07F7B9E7E6
:102DA8002027F5E792FAA2F242B1B2FA82F2013292
:102DB80002F01F0202EB42021205B5E72022F6E7F5
:102DC800D6B9940E0134A40604F0F84406BB970E55
:102DD800013707F01F0C012707FA0CF73C4336BBF5
:102DE800920E013202F01F0202EB42021E3A120555
:102DF80042F00072224398E792FAA2F434B1B4FA8E
:102E080084F40134A40604F0F844DFE72024F8E74A
:102E180092FAA2F74FB1B7FA87F7013707F01F0701
:102E28004FF0010C0CFA07F7D8E72027F5E792FADC
:102E3800A2F25AB1B2FA82F2013202F01F0202EB98
:102E480042021E3A120542F00072D3E72022F3E74D
:102E580011F4000F7FF417AF1A68B2F1A04F7FF496
:102E68001AAF44F4000420498A6822F0E07214433F
:102E78008C601E4A126892091D49A1FB0212920930
:102E880002EB420292001832019202E0019A013AE2
:102E98000192019A002AF9D1FDE611F0807F7FF4B2
:102EA800F6AE1968134A91423FF4F5AE44F08074C7
:102EB8000D498A6822F0E07214438C60EBE611F445
:102EC800800F7FF4E8AE19680A4A91423FF4E3AEF6
:102ED80044F4800404498A6822F0E07214438C6048
:102EE800D9E60220DAE600BF000300500400002003
:102EF800632D3E050001005090F85820012A7FD02C
:102F080010B49DB00346012280F858200022189280
:102F180019920068B0F1A04F39D000220192019AAD
:102F2800002A37D0926812F0040200D0012280688B
:102F380010F0040F54D1002A52D10A68002A32D066
:102F4800304CA26822F46042486893F838C040EADE
:102F58004C300243A2604FF0A042926812F0010286
:102F680000D001222848806810F0010000D001201C
:102F7800024341D1234CA26822F4716222F00F026D
:102F88000868896801430A43A26000202DE01E4AB0
:102F98000192C4E7DA6D42F02002DA65002283F874
:102FA8005820012024E017498A6822F460428A6088
:102FB8004FF0A042926812F0010200D0012212499B
:102FC800896811F0010100D001210A4316D10D4989
:102FD8008A6822F4716222F00F028A60002004E0FD
:102FE800DA6D42F02002DA650120002283F85820C9
:102FF8001DB05DF8044B70470020F6E70020F4E7A9
:10300800022070470003005000010050074AD368AF
:1030180023F4E0631B041B0C000200F4E06003438C
:1030280043F0BF6343F40033D360704700ED00E022
:1030380000B5194BDB68C3F30223C3F1070CBCF1DD
:10304800040F28BF4FF0040C03F1040EBEF1060F65
:1030580018D9033B4FF0FF3E0EFA0CFC21EA0C0195
:1030680099400EFA03F322EA0303194300280BDB05
:103078000901C9B200F1604000F5614080F8001311
:103088005DF804FB0023E5E700F00F000901C9B271
:10309800024B1954F4E700BF00ED00E014ED00E026
:1030A800002807DB00F01F02400901239340024A71
:1030B80042F82030704700BF00E100E00138B0F16D
:1030C800807F0BD24FF0E0235861054AF02182F847
:1030D80023100020986107221A6170470120704769
:1030E80000ED00E030B4C46C056D6560446D14B14A
:1030F800846DC56D6560446C04F01F0C012404FAEE
:103108000CF4056C6C60046863608368102B05D050
:10311800036899600368DA6030BC704703689A6096
:103128000368D960F8E7000003680C4A934213D893
:103138000B49DBB2083B0B4AA2FB0323426C22F08B
:1031480003020A448264084AC264C3F304130122D6
:1031580002FA03F3036570470449EAE707040240EB
:1031680000080240CDCCCCCC8008024020080240A8
:103178000379074A1A4492004265064A8265013B70
:1031880003F01F03012202FA03F3C365704700BF6F
:103198003F8200104009024000285BD010B5044669
:1031A80001682D4B99423DD82C4B0B442C4AA2FB6D
:1031B80003231B099B0043642A4B0364022384F8FE
:1031C80025300A6822F4FF4222F07002A368E06802
:1031D80003432069034360690343A0690343E0692B
:1031E8000343206A034313430B602046FFF79CFF09
:1031F800A368B3F5804F20D0A36C22791A60E36CE2
:10320800226D5A606368013B032B19D9002363655B
:10321800A365E3650020E063012384F8253084F882
:10322800240010BD104B0B440D4AA2FB03231B09BD
:103238009B0043640D4B0364C0E700236360DBE736
:103248002046FFF795FF636D00221A60A36DE26DBB
:103258005A60DFE70120704707040240F8FFFDBF0E
:10326800CDCCCCCC00000240F8FBFDBF00040240EE
:1032780038B5044690F82400012841D0012084F88C
:10328800240094F82500C0B2012804D0002384F853
:103298002430022038BD022084F825000020E06395
:1032A8002568286820F0010028602046FFF71AFFEB
:1032B800236BD3B12268136843F00E031360A36C29
:1032C8001A6812F4803F03D01A6842F480721A60B8
:1032D800636D1BB11A6842F480721A602268136821
:1032E80043F0010313600020D4E72268136823F039
:1032F800040313602268136843F00A031360DEE7CF
:103308000220C7E738B5036C196804682568436C60
:1033180003F01F0304229A400A4215D015F0040F47
:1033280012D0236813F0200F03D1236823F004037D
:103338002360436C03F01F02016C042393404B602D
:10334800036B03B1984738BD02229A400A421CD049
:1033580015F0020F19D0236813F0200F06D1236847
:1033680023F00A032360012380F82530436C03F01F
:103378001F02016C022393404B60002380F8243025
:10338800C36A002BDFD09847DDE7082202FA03F36F
:103398000B42D8D015F0080FD5D0236823F00E03C0
:1033A8002360436C03F01F03016C012202FA03F34C
:1033B8004B60C26380F82520002380F82430436BDB
:1033C800002BC0D09847BEE7F0B583B0002362E079
:1033D80085685E000324B44025EA0405CC68B4403F
:1033E8002C438460446824EA0C0C4C68C4F3001431
:1033F8009C4044EA0C0444605EE0DD08083550F85F
:10340800256003F007044FEA840C0F2404FA0CF437
:1034180026EA040E0C6904FA0CF444EA0E0440F897
:10342800254060E0052400E0002404FA0EF42C4353
:103438000CF1020C554D45F82C40554CA568D44369
:1034480025EA02064F6817F4801F01D042EA0506F4
:103458004F4DAE60ED6804EA05064F6817F4001F8B
:1034680001D042EA05064A4DEE606D6804EA050699
:103478004F6817F4003F01D042EA0506444D6E60DC
:103488002D682C404E6816F4803F01D042EA0504AE
:103498003F4A146001330A6832FA03F474D04FF0DB
:1034A800010C0CFA03FC1CEA0202F3D04C6804F08D
:1034B8000304013C012C8BD94C6804F00304032C51
:1034C8000CD0C4685D004FF0030C0CFA05FC24EA2C
:1034D8000C0C8C68AC4044EA0C04C4604C6804F0E2
:1034E8000304022C89D004684FEA430E4FF0030C02
:1034F8000CFA0EFC24EA0C0C4C6804F0030404FAE1
:103508000EF444EA0C0404604C6814F4403FC1D043
:10351800204C256E45F001052566246E04F0010453
:103528000194019C4FEA930C0CF10205174C54F8D6
:10353800255003F003044FEA840E0F2404FA0EF416
:1035480025EA0405B0F1904F3FF46EAF124CA0424B
:1035580012D004F58064A04210D004F58064A04223
:103568000ED004F58064A0420CD004F58064A0421B
:103578003FF458AF062458E7012456E7022454E7DD
:10358800032452E7042450E703B0F0BD00000140D3
:103598000004014000100240000400480AB18161A3
:1035A800704781627047002859D010B5044690F8DA
:1035B8004130002B43D0242384F84130226813681B
:1035C80023F0010313606368226823F070631361BA
:1035D8002268936823F400439360E368012B33D097
:1035E800A368226843F404439360E368022B31D054
:1035F8002268536843F0007343F400435360226821
:10360800D36823F40043D360236962691343A16933
:10361800226843EA0123D360E369216A22680B43E5
:1036280013602268136843F001031360002060648C
:10363800202384F84130206384F8420010BD80F8CC
:103648004030FDF79FFEB6E7A368226843F40043C5
:103658009360CAE723684FF400625A60C8E7012004
:10366800704790F84130DBB2202B24D190F84030DD
:10367800012B22D0012380F84030242380F84130E8
:103688000268136823F0010313600268136823F4C7
:103698008053136002681368194311600268136845
:1036A80043F001031360202380F84130002380F8A1
:1036B800403018467047022070470220704790F843
:1036C8004130DBB2202B22D190F84030012B20D0A2
:1036D800012380F84030242380F8413002681368C1
:1036E80023F0010313600268136823F4706343EA4C
:1036F800012111600268136843F00103136020235D
:1037080080F84130002380F8403018467047022086
:103718007047022070470000002800F0868010B52E
:1037280082B0044690F83A30DBB2052B7FD090F88F
:103738003A30DBB2022B7CD03F4B1A6E42F00102CA
:103748001A661B6E03F001030193019B90F83A304F
:103758000BB980F839302046FDF700FFA368402BED
:1037680025D0602B23D02268136823F01003E16A68
:103778000B43136021680B68304A1A406368A068DD
:103788000343E068034320690343207D012849D0AF
:1037980000200343606A0343A06A0343206B43EAA3
:1037A800C043606B43EA006313430B6020E0226868
:1037B800136823F01003E16A0B43136021680B6858
:1037C8001E4A1A406368A068034320690343207DAA
:1037D800012824D000200343606A0343A06A0343FE
:1037E800206B43EAC043606B43EA006313430B60FA
:1037F80021688B69002B09DB8B6923F03F03A269E1
:10380800E0690243206A024313438B6194F83A301B
:1038180013B9012384F83A30002002B010BD4FF4E8
:103828008070D8E74FF48070B3E70120704701201B
:10383800F3E70120F1E700BF00100240113E00E06D
:10384800A8B190F83A30DBB2052B12D090F83A3094
:10385800DBB2012B01D00120704701680B6843F0EF
:1038680001030B60042380F83A30002070470120E0
:1038780070470120704738B512F4804F43D0046870
:10388800B4F8503091F800C04FEACC0E1EFA83F31A
:103898002344B3F80244C4F309048B69A34228D330
:1038A8001B1B8B618B697BB9056835F82C309BB283
:1038B80023F4804323F0700383F4005343F400435C
:1038C80043F0800325F82C3012F0400F0ED0026828
:1038D8000D7832F825309BB223F4E04323F07003CF
:1038E80043F4004343F0C00322F8253024B92046AE
:1038F80038BD00238B61D5E723460A8949690068EA
:1039080003F014FCF3E70468B4F8503091F800C0F1
:103918004FEACC0E1EFA83F32344B3F80644C4F3EB
:1039280009048B69A3422FD31B1B8B618B697BB95D
:10393800056835F82C309BB223F4804323F07003DC
:1039480083F4005343F4004343F0800325F82C30FC
:1039580012F0400F0FD1026891F800C032F82C30F5
:103968009BB223F4E04323F0700343F4004343F095
:10397800C00322F82C30002CB9D023464A89496963
:10398800006803F0D3FBB2E700238B61CEE7002881
:103998006DD030B587B0044690F8A9323BB1032307
:1039A80084F8A932206802F09FFC00231FE080F809
:1039B800A83204F0B7FBF2E75A1C02EB820104EBD1
:1039C800C1010120487002EB820104F8313003EB99
:1039D800830104EBC101CB8602EB820C04EBCC0C17
:1039E80000208CF803008863C8630864D3B2606859
:1039F8008342E1D3002316E003EB830204EBC20207
:103A0800002182F8691182F8683182F86B11C2F8D6
:103A18007811C2F87C1103EB830204EBC202C2F8EE
:103A280080110133DBB29842E6D8A4465CF8105BFB
:103A3800EE46BCE80F00AEE80F00DCF80030CEF828
:103A48000030231D0ECB284602F058FC002384F8D2
:103A58002430012384F8A932E369012B02D0002025
:103A680007B030BD204600F0E8FE0020F8E701204E
:103A7800704790F8A832012B0ED010B504460123E8
:103A880080F8A832006802F026FC206802F07BFF6C
:103A9800002084F8A80210BD0220704770B50546C2
:103AA8000C46164612F0400F00F009810268B2F881
:103AB80050300978C80010FA83F31344B3F802248D
:103AC800C2F30902A369934251D99B1AA361A3695E
:103AD800002B68D16378002B4CD12A68B2F850309B
:103AE80012FA83F30344B3F8022492B222F4F842A0
:103AF80092B2A3F80224B3F802246FEA42426FEAB2
:103B0800524292B2A3F8022429686278002A3DD171
:103B1800B1F8503011FA83F3227803EBC203B3F8FB
:103B2800062492B222F4F84292B2A3F80624B3F81B
:103B380006246FEA42426FEA524292B2A3F8062480
:103B48002178284604F032FB16F4804F40D02A68CA
:103B5800217832F821309BB223F4E04323F070033C
:103B680043F4404343F0800322F8213030E000233F
:103B7800A361ACE7012BC7D12A68B2F8503012FA1A
:103B880083F303440022A3F80224BDE7012AD7D116
:103B9800B1F8503011FA83F3217803EBC103002206
:103BA800A3F80624CCE716F4804F0DD0286830F827
:103BB80021309BB223F4E04323F0700343F44043E5
:103BC80043F0800320F8213094F82430012B12D0E0
:103BD8002A68217832F821309BB223F4E04323F09D
:103BE800400383F0300343F4004343F0800322F89A
:103BF8002130002070BD636913446361E369134495
:103C0800E361216A236999421BD3C91A2162627848
:103C1800002A3FD12968B1F8502011FA82F22178A0
:103C280002EBC1023E2B18D9590913F01F0F00D11E
:103C380001396FEAC1616FEA514189B2A2F80214F1
:103C48002AE021B9002384F824301346DFE7002353
:103C580084F8243023620B46D9E78BB9B2F80214F2
:103C680089B221F4F84189B2A2F80214B2F8021418
:103C78006FEA41416FEA514189B2A2F802140BE0A0
:103C8800590813F0010F00D00131890289B2A2F856
:103C9800021401E0012A06D09BB2228961692868D2
:103CA80002F080FE94E72968B1F8502011FA82F2F8
:103CB800217802EBC10299B2A2F80214ECE702687B
:103CC800B2F850300978C80010FA83F31344B3F8F7
:103CD8000624C2F30902A369934252D39B1AA36133
:103CE800A369002B69D16378002B4DD12A68B2F8FB
:103CF800503012FA83F31844B0F802349BB223F41C
:103D0800F8439BB2A0F80234B0F802346FEA434398
:103D18006FEA53439BB2A0F8023429686278002AFC
:103D28003ED1B1F8503011FA83F3227803EBC20385
:103D3800B3F8062492B222F4F84292B2A3F8062409
:103D4800B3F806246FEA42426FEA524292B2A3F8ED
:103D580006242178284604F029FA16F4804F7FF4C7
:103D680037AF2A68217832F821309BB223F4E04338
:103D780023F0700343F4404343F0800322F82130DA
:103D880026E70023A361ABE7012BC6D12A68B2F866
:103D9800503012FA83F318440023A0F80234BCE729
:103DA800012AD6D1B1F8503011FA83F3217803EB08
:103DB800C1030022A3F80624CBE716F4804F0DD1E7
:103DC800286830F821309BB223F4E04323F07003D5
:103DD80043F4404343F0800320F8213094F8243022
:103DE800012B7FF4F5AE636913446361E3691344FF
:103DF800E361216A236999421BD3C91A21622968A0
:103E08006278002A3ED1B1F8502011FA82F2217866
:103E180002EBC1023E2B18D9590913F01F0F00D12C
:103E280001396FEAC1616FEA514189B2A2F80614FB
:103E38002AE021B9002384F824301346DFE7002361
:103E4800236284F824300B46D9E78BB9B2F80614FC
:103E580089B221F4F84189B2A2F80614B2F806141E
:103E68006FEA41416FEA514189B2A2F806140BE0AA
:103E7800590813F0010F00D00131890289B2A2F864
:103E8800061401E0012A06D09BB26289616928689C
:103E980002F088FD9CE6B1F8502011FA82F22178F0
:103EA80002EBC10299B2A2F80614EDE72DE9F04140
:103EB8000546CAE003889BB223F4E14323F070036C
:103EC8006FEA43436FEA53439BB203802968B1F812
:103ED800503095F82820D20012FA83F30B44B3F837
:103EE8000234C3F309036B64EA6B1344EB630021E8
:103EF800284604F05BF995F82430002B00F0A580E3
:103F08002B6C002B40F0A18095F824302A6843F0F0
:103F18008003A2F84C30002385F8243095E0B0F8EF
:103F2800503095F86821D20012FA83F30344B3F8AD
:103F38000634C3F30903C5F88431B5F86E2105F5D5
:103F48002C7103F0F3F82A68138823F070031B051B
:103F58001B0D43F080031380284604F013F974E026
:103F680089B9B3F8062492B222F4F84292B2A3F8BF
:103F78000624B3F806246FEA42426FEA524292B22C
:103F8800A3F80624BFE04A0811F0010F00D001325F
:103F9800920292B2A3F80624B5E030F824309EB21B
:103FA80013F4004F40F0BE8016F0800F4DD0621C15
:103FB80002EB820105EBC101286830F824309BB27E
:103FC80023F4E14323F070036FEA43436FEA53435A
:103FD8009BB220F82430CB78022B00F0A78104EBA9
:103FE800840305EBC30300221A6493F8343023B327
:103FF80016F0400F00F063814B78002B40F04C81A5
:104008002A68B2F8503012FA83F3621C02EB82027B
:1040180015F8322003EBC203B3F8022492B222F45B
:10402800F84292B2A3F80224B3F802246FEA42429B
:104038006FEA524292B2A3F80224013404EB8404DA
:1040480015F83410284604F0B1F82868B0F8443060
:1040580013F4004F00F0AE81B0F84440A3B214F05E
:104068000F049AD113F0100F3FF424AF03889AB2CB
:1040780013F4006F7FF453AF12F4004FE5D00388B8
:1040880023F070031B051B0D43F080030380286891
:10409800B0F8503095F86821D20012FA83F303443F
:1040A800B3F80634C3F30903C5F884318BB1D5F8E6
:1040B8007C1171B1B5F86E2103F038F8D5F8842178
:1040C800D5F87C311344C5F87C310021284604F02A
:1040D80061F82B681A8812F4006FB6D1B3F8502033
:1040E80013FA82F3D5F878113E297FF639AF4A09D9
:1040F80011F01F0F00D1013A6FEAC2626FEA524213
:1041080092B2A3F806242A6813889BB223F480434A
:1041180023F0700383F4405343F4004343F08003D7
:10412800138092E730F8243023F070031B051B0D31
:1041380043F0800320F8243004EB8401C90001F522
:10414800B47105EB010804EB840305EBC30393F892
:104158007431002B40D12868B0F8503004EB840249
:1041680005EBC20292F86821D20012FA83F30344E5
:10417800B3F80674C7F3090717BB04EB840305EB10
:10418800C303D3F884213A44C3F88421D3F87C21AB
:104198003A44C3F87C21D3F880313BB104EB840363
:1041A80005EBC303D3F878319F4270D204EB840344
:1041B80005EBC30393F86811284603F0EBFFF3E619
:1041C80004EB840105EBC1013B46B1F86E21D1F83F
:1041D8007C1102F0ABFFD0E704EB840305EBC303CB
:1041E80093F86B31022B33D0296804EB840205EB7A
:1041F800C20292F8680131F820309BB223F4E04300
:1042080023F0700343F4004343F0C00321F8203047
:10421800286892F8683130F8232012F4804F1ED0B5
:10422800B0F85020DB0013FA82F30344B3F80274A9
:10423800C7F30907002FA0D004EB840105EBC101E7
:104248003B46B1F87021D1F87C1102F06FFF94E77A
:10425800324641462846FFF70EFB07468DE7B0F881
:104268005020DB0013FA82F30344B3F80674C7F353
:104278000907002F81D004EB840105EBC1013B46FF
:10428800B1F87221D1F87C1102F050FF75E7414670
:10429800286802F09BFB87E6012B7FF4CEAE2A68E4
:1042A800B2F8503012FA83F3621C02EB820215F85E
:1042B800322003EBC2030022A3F80224BDE62968DA
:1042C800631C03EB830305EBC3035A78E2B9B1F827
:1042D800503011FA83F3621C02EB820215F8322087
:1042E80003EBC203B3F8062492B222F4F84292B266
:1042F800A3F80624B3F806246FEA42426FEA524252
:1043080092B2A3F8062498E6012A7FF496AEB1F893
:10431800503011FA83F3621C02EB820215F8322046
:1043280003EBC2030022A3F8062486E616F4807F76
:104338003BD12868B0F85030621C02EB820215F8B5
:104348003260F20012FA83F30344B3F80234C3F381
:10435800090304EB840205EBC202126C9A4210D9DD
:1043680004EB840705EBC707D21A3A6404EB84020E
:1043780005EBC202126C5AB93146284603F016FF03
:1043880063E604EB840205EBC20200271764EDE73D
:1043980004EB840205EBC202D66B1E44D663546C50
:1043A8002344536402F012FB4FE632462846FFF7D7
:1043B80075FB4AE60020BDE8F08190F8A832012B91
:1043C8000DD010B50446012380F8A83280F82410D7
:1043D800006802F0D2FA002084F8A80210BD02207A
:1043E800704710B50446006802F0D8FA10F4004F80
:1043F80023D110F4806F24D110F4804F32D110F4FF
:10440800005F39D110F4805F40D110F4006F67D19C
:1044180010F0800F40F0818010F4007F40F0AD80F4
:1044280010F4807F27D02268B2F844309BB223F47E
:1044380080739BB2A2F844301DE02046FFF736FD9A
:1044480019E02268B2F844309BB223F480639BB22F
:10445800A2F84430204603F0BAFE00212046FFF7B8
:10446800ACFF08E02268B2F844309BB223F48043E2
:104478009BB2A2F8443010BD2268B2F844309BB217
:1044880023F400539BB2A2F84430F4E72268B2F850
:1044980040309BB223F004039BB2A2F8403022685C
:1044A800B2F840309BB223F008039BB2A2F8403028
:1044B80094F8E032012B0CD0204603F0ABFE2268C2
:1044C800B2F844309BB223F480539BB2A2F8443034
:1044D800D1E7002184F8E012204603F053FFEBE710
:1044E8002268B2F840309BB243F00803A2F840308B
:1044F8002268B2F844309BB223F400639BB2A2F85E
:1045080044302268B2F840309BB243F00403A2F86A
:104518004030204603F06EFEADE72268B2F8443022
:104528009BB223F080039BB2A2F8443094F8E032A7
:10453800FBB92268B2F840309BB243F00403A2F8FA
:1045480040302268B2F840309BB243F00803A2F82A
:104558004030012184F8E0122368B3F85430C3F3E3
:104568008D0303F03C03C4F8E432204603F00AFF4D
:1045780081E7204603F03EFE7DE72268B2F844302A
:104588009BB223F400739BB2A2F84430204603F098
:1045980018FE70E710B504468C4611F0800F2AD13A
:1045A80001F0070000EB8001C90001F5B47E04EBBF
:1045B8000E0100EB800004EBC0004FF0000E80F805
:1045C80069E10CF0070C81F800C00A61CB704A78E9
:1045D8000AB1A1F80EC0022B19D094F8A832012B09
:1045E80018D0012384F8A832206801F098FE002032
:1045F80084F8A80210BD01F00700013000EB80012B
:1046080004EBC1014FF0010E81F801E0D9E7002366
:104618000B71E2E70220EDE710B504460B4611F0F6
:10462800800F1FD101F0070202EB8201C90001F5DA
:10463800B471014402EB820200EBC202002082F84E
:10464800690103F007030B7094F8A832012B13D00B
:10465800012384F8A832206802F02EF8002084F89C
:10466800A80210BD01F00702013202EB820100EB43
:10467800C10101204870E4E70220F2E710B501F01B
:10468800070404EB8401C90001F5B471014404EB8B
:10469800840C00EBCC0CCCF87C21CCF880310023C6
:1046A800CCF884318CF869318CF8684124B90068F9
:1046B80002F08CF9002010BD006802F087F9F9E7D4
:1046C80001F0070101EB810100EBC101D1F8840180
:1046D800704710B501F0070404F1010C0CEB8C01D4
:1046E80000EBC10104EB840E00EBCE0ECEF83C20AB
:1046F800CEF8403001228EF84C20CEF84830002306
:10470800CEF844304A700CEB8C0C00F83C4024B9CD
:10471800006802F05BF9002010BD006802F056F94D
:10472800F9E70B4601F0070241688A422AD810B51A
:10473800044613F0800F1DD103EB8301C90001F576
:10474800B471014403EB830300EBC303002083F837
:10475800690101238B700A7094F8A832012B13D0D9
:10476800012384F8A832206802F091F8002084F828
:10477800A80210BD531C03EB830100EBC10101200B
:104788004870E6E7012070470220F2E70B4601F087
:104798000F014268914230D810B5044613F0800FDB
:1047A80021D103F0070202EB8201C90001F5B471BF
:1047B800014402EB820200EBC202002082F8690188
:1047C80000228A7003F007030B7094F8A832012BBB
:1047D80015D0012384F8A832206802F07DF8002063
:1047E80084F8A80210BD03F00702013202EB82012F
:1047F80000EBC10101204870E2E701207047022068
:10480800F0E711F0800F0BD001F00701013101EB47
:10481800810100EBC10152B90A73CB8000207047B7
:1048280001EB8101C90001F5B4710144F3E70122EC
:104838000A730B811B0C4B81F0E7034602680121C8
:10484800C0F8E812002083F8E002B2F854309BB2B6
:104858000B43A2F85430B2F854309BB243F0020331
:10486800A2F8543070470000002836D13E4B1B6830
:1048780003F4C063B3F5806F08D03B4AD2F88030A8
:1048880023F48073C2F8803000207047364AD2F88B
:10489800803023F48073C2F88030136823F4C06337
:1048A80043F400731360314B1B68322202FB03F39D
:1048B8002F4AA2FB03239B0C013300E0013B2A4A49
:1048C800526912F4806F01D0002BF7D1264B5B6937
:1048D80013F4806F44D100207047B0F5007F08D0F2
:1048E800214A136823F4C06343F4806313600020F3
:1048F80070471D4B1B6803F4C063B3F5806F08D085
:10490800194AD2F8803043F48073C2F8803000200E
:104918007047154AD2F8803043F48073C2F880306B
:10492800136823F4C06343F4007313600F4B1B68D0
:10493800322202FB03F30E4AA2FB03239B0C013332
:1049480000E0013B084A526912F4806F01D0002B45
:10495800F7D1054B5B6913F4806F03D100207047D2
:1049680003207047032070470070004004000020B7
:1049780083DE1B43024A936843F480439360704785
:1049880000700040124BDA6802F00302D868C0F3E6
:104998000310431C032A11D00E48B0FBF3F00C4B54
:1049A800DB68C3F3062303FB00F0094BDB68C3F3A2
:1049B800416301335B00B0FBF3F070470648B0FB7E
:1049C800F3F0034BDB68C3F3062303FB00F0ECE7CB
:1049D800001002400024F40000366E01002800F0A8
:1049E800548270B582B00446036813F0010F37D0C3
:1049F800A44A936803F00C03D26802F003020C2B5C
:104A080023D0082B23D06368B3F5803F4ED0B3F58D
:104A1800A02F51D09B4B1A6822F480321A601A6872
:104A280022F480221A606368002B52D0FDF720F828
:104A38000546944B1B6813F4003F11D1FDF718F895
:104A4800401B6428F5D9032028E2032AD9D18D4BCD
:104A58001B6813F4003F03D06368002B00F0178233
:104A6800236813F0020F5DD0864A936803F00C03A5
:104A7800D26802F003020C2B3AD0042B3AD0E36838
:104A8800002B75D07F4A136843F480731360FCF7DA
:104A9800EFFF05467B4B1B6813F4806F5FD1FCF773
:104AA800E7FF401B0228F5D90320F7E1754A136890
:104AB80043F480331360B6E703F18043A3F53C3336
:104AC8001A6842F480221A601A6842F480321A6026
:104AD800A9E7FCF7CDFF05466A4B1B6813F4003FB6
:104AE800BED0FCF7C5FF401B6428F5D90320D5E1EB
:104AF800022AC2D1634B1B6813F4806F03D0E368AA
:104B0800002B00F0C6815F4A536823F0FE432169F9
:104B180043EA016353605C4B1868FCF765FF0028A3
:104B280040F0B981236813F0080F4CD063699BB338
:104B3800544AD2F8943043F00103C2F89430FCF799
:104B480097FF05464F4BD3F8943013F0020F3AD134
:104B5800FCF78EFF401B0228F4D903209EE1494A46
:104B6800536823F0FE43216943EA01635360D9E7A0
:104B7800444A136823F480731360FCF779FF0546F1
:104B8800404B1B6813F4806FCCD0FCF771FF401BBF
:104B98000228F5D9032081E13A4AD2F8943023F06B
:104BA8000103C2F89430FCF763FF0546354BD3F890
:104BB800943013F0020F06D0FCF75AFF401B02286E
:104BC800F4D903206AE1236813F0040F00F0818010
:104BD8002C4B9B6D13F0805F36D12A4B9A6D42F0B7
:104BE80080529A659B6D03F080530193019B0125C8
:104BF800264B1B6813F4807F28D0A368012B39D07B
:104C0800052B45D01F4BD3F8902022F00102C3F8A2
:104C18009020D3F8902022F00402C3F89020A368D3
:104C2800002B43D0FCF724FF0646164BD3F89030F0
:104C380013F0020F4CD1FCF71BFF801B41F28833A5
:104C48009842F2D9032029E10025D1E70F4A1368D9
:104C580043F480731360FCF70BFF06460B4B1B688D
:104C680013F4807FC9D1FCF703FF801B0228F5D914
:104C7800032013E1034AD2F8903043F00103C2F84D
:104C88009030CCE7001002400C000020007000407B
:104C98008A4BD3F8902042F00402C3F89020D3F84E
:104CA800902042F00102C3F89020B8E7FCF7E0FE3C
:104CB8000646824BD3F8903013F0020F08D0FCF769
:104CC800D7FE801B41F288339842F2D90320E5E0F1
:104CD800E5B9236813F0200F35D0A369E3B1774A0B
:104CE800D2F8983043F00103C2F89830FCF7C0FEC0
:104CF8000546724BD3F8983013F0020F23D1FCF716
:104D0800B7FE401B0228F4D90320C7E06B4A936D15
:104D180023F080539365DCE7684AD2F8983023F093
:104D28000103C2F89830FCF7A3FE0546634BD3F89D
:104D3800983013F0020F06D0FCF79AFE401B0228A9
:104D4800F4D90320AAE0E369002B00F0A6805B4AAF
:104D5800926802F00C020C2A69D0022B1DD0574B26
:104D68001A6822F080721A60DA6822F00302DA60A8
:104D7800DA6822F0887222F48032DA60FCF778FE72
:104D880004464E4B1B6813F0007F4ED0FCF770FEB4
:104D9800001B0228F5D9032080E0484A136823F055
:104DA80080731360FCF764FE0546444B1B6813F0E0
:104DB800007F06D0FCF75CFE401B0228F5D90320D3
:104DC8006CE03E4AD3683E491940236A606A01385C
:104DD80043EA0013A06A43EA0023206B4008013825
:104DE80043EA4053606B4008013843EA4063E06A95
:104DF80043EAC0630B43D360136843F080731360C6
:104E0800D36843F08073D360FCF732FE04462B4B23
:104E18001B6813F0007F06D1FCF72AFE001B02284E
:104E2800F5D903203AE0002038E0002036E0012BD5
:104E380036D0224BDB6803F00301226A914231D15C
:104E480003F0F002616A0139B2EB011F2CD103F4BF
:104E5800FE42A16AB2EB012F28D103F07842E16A41
:104E6800B2EBC16F24D103F4C001226B5208013A9E
:104E7800B1EB425F1ED103F0C063626B5208013A86
:104E8800B3EB426F18D1002008E0012070470120E1
:104E980004E0012002E0012000E0002002B070BD23
:104EA8000120FBE70120F9E70120F7E70120F5E7FA
:104EB8000120F3E70120F1E70120EFE700100240AD
:104EC8000C809F011E4B9B6803F00C03042B33D00E
:104ED8001B4B9B6803F00C03082B2FD0184B9B68C7
:104EE80003F00C030C2B01D000207047144BDA6838
:104EF80002F00302D868C0F30310431C032A11D040
:104F08001048B0FBF3F00E4BDB68C3F3062303FB3A
:104F180000F00B4BDB68C3F3416301335B00B0FB6C
:104F2800F3F070470848B0FBF3F0054BDB68C3F3B8
:104F3800062303FB00F0ECE702487047024870477D
:104F4800001002400024F40000366E01002800F032
:104F5800E680F8B50C460546744B1B6803F00F0352
:104F68008B420BD2714A136823F00F030B43136073
:104F7800136803F00F038B4240F0D3802E6816F0BD
:104F880001065FD06B68032B2FD0022B4DD0684BE6
:104F98001B6813F4806F00F0C680FFF793FF654B22
:104FA80098424DD9624A936823F0F00343F0800396
:104FB800936080265E4A936823F0030369680B4375
:104FC8009360FCF755FD0746594B9B6803F00C03AB
:104FD8006A68B3EB820F35D0FCF74AFDC01B41F27B
:104FE80088339842F0D9032078E0514B1B6813F0BE
:104FF800007F01D1012071E0FFF7C4FC4D4B9842BE
:105008001AD94B4B9B6813F0F00F05D02E6816F099
:105018000206CFD0AB688BB9454A936823F0F003FA
:1050280043F0800393608026C4E7414B1B6813F468
:10503800003FB2D1012051E00026BBE70026B9E7C6
:105048000026B7E72B6813F0020F48D013F0040FBF
:1050580004D0374A936843F4E06393602B6813F0F5
:10506800080F06D0324A936823F47C5343F4E06374
:1050780093602F4A936823F0F003A9680B43936069
:105088002A4B1B6803F00F03A34230D82B6813F098
:10509800040F06D0264A936823F4E063E9680B43BB
:1050A80093602B6813F0080F07D0214A936823F404
:1050B8006053296943EAC1039360FFF703FF1C4B60
:1050C8009B68C3F303131C4AD35C03F01F03D84047
:1050D8001A4B18601A4B1868FCF786FCF8BD802E2E
:1050E800CED1134A936823F0F0039360C8E70F4AC0
:1050F800136823F00F0323431360FCF7B9FC06463B
:105108000A4B1B6803F00F03A342BFD0FCF7B0FCA7
:10511800801B41F288339842F2D90320DEE7012050
:1051280070470120DAE70120D8E700BF00200240DD
:105138000010024000B4C4042492000804000020B7
:105148000C000020024A136843F4002313607047E0
:10515800001002407047000008B5064BDB6913F4E5
:10516800807F00D108BDFFF7F5FF024B4FF4807236
:105178001A62F7E700100240F0B583B004460368EE
:1051880013F4002F69D0AE4B9B6D13F0805F1ED1D6
:10519800AB4B9A6D42F080529A659B6D03F0805339
:1051A8000193019B0126A74A136843F48073136097
:1051B800FCF75EFC0546A34B1B6813F4807F08D1FF
:1051C800FCF756FC401B0228F5D9032502E000260F
:1051D800E9E7002545BB9A4BD3F8903013F44073A8
:1051E80015D0226C9A4212D0954AD2F8903023F406
:1051F8004073D2F8901041F48031C2F89010D2F880
:10520800901021F48031C2F89010C2F8903013F059
:10521800010F10D145B98A4AD2F8903023F440736F
:10522800216C0B43C2F89030C6B1854A936D23F0C8
:105238008053936512E0FCF71BFC0746804BD3F8BC
:10524800903013F0020FE5D1FCF712FCC01B41F2BD
:1052580088339842F2D90325DCE70025236813F048
:10526800010F08D0764AD2F8883023F0030361682A
:105278000B43C2F88830236813F0020F08D0704A35
:10528800D2F8883023F00C03A1680B43C2F88830A9
:10529800236813F0040F08D0694AD2F8883023F045
:1052A8003003E1680B43C2F88830236813F0080F15
:1052B80008D0634AD2F8883023F0C00321690B4331
:1052C800C2F88830236813F0200F08D05C4AD2F85F
:1052D800883023F4406361690B43C2F8883023683F
:1052E80013F0400F08D0564AD2F8883023F44053C0
:1052F800A1690B43C2F88830236813F0800F08D0E7
:105308004F4AD2F8883023F44043E1690B43C2F88E
:105318008830236813F4807F08D0494AD2F888304F
:1053280023F44033216A0B43C2F88830236813F40E
:10533800007F08D0424AD2F8883023F44023616ABB
:105348000B43C2F88830236813F4806F0CD03C4AB2
:10535800D2F8883023F44013A16A0B43C2F888308E
:10536800A36AB3F5801F57D0236813F4006F0CD0DD
:10537800334AD2F8883023F44003E16A0B43C2F879
:105388008830E36AB3F5800F4BD0236813F4805F4D
:105398000CD02B4AD2F8883023F04073216B0B4392
:1053A800C2F88830236BB3F1807F3FD0236813F4B1
:1053B800005F0CD0224AD2F8883023F04063616B3A
:1053C8000B43C2F88830636BB3F1006F33D02368A6
:1053D80013F4804F0CD01A4AD2F8883023F0406377
:1053E800A16B0B43C2F88830A36BB3F1006F2BD0CD
:1053F800236813F4004F0CD0114AD2F8883023F0F8
:105408004053E16B0B43C2F88830E36BB3F1805F24
:105418001FD0284603B0F0BDD36843F48013D3608F
:10542800A2E7D36843F48013D360AEE7D36843F4AC
:105438008013D360BAE7D36843F48013D360C6E718
:105448000010024000700040D36843F48013D3601A
:10545800CEE7D36843F48033D360DAE700286FD00F
:1054680010B50446436A33B94368B3F5827F05D063
:105478000023C36102E00023036143610023A362A8
:1054880094F85D30002B52D0022384F85D302268F6
:10549800136823F040031360E368B3F5E06F4CD959
:1054A8000022B3F5706F04D0B3F5E06F01D000238C
:1054B800A362636803F48273A16801F404410B4397
:1054C800216901F002010B43616901F001010B43FD
:1054D800A16901F400710B43E16901F038010B4344
:1054E800216A01F080010B43A16A01F40051206890
:1054F8000B430360638B03F00403616A01F010013E
:105508000B43616B01F008010B43E16801F4706122
:105518000B43216813434B602268D36923F400636B
:10552800D36100202066012384F85D3010BD84F823
:105538005C302046FCF7A8F8A6E74FF48052B0E7A5
:105548000120704730B4036A23F001030362036A41
:105558004568826922F4803222F073020C68224383
:1055680023F002038C6823431D4CA0420FD004F59E
:105578000064A0420BD004F54064A04207D004F5B3
:105588008064A04203D004F58064A04205D123F0D2
:105598000803CC68234323F00403114CA0420FD026
:1055A80004F50064A0420BD004F54064A04207D083
:1055B80004F58064A04203D004F58064A04207D1BA
:1055C80025F4407C4C6944EA0C0C8D6945EA0C05CD
:1055D800456082614A684263036230BC704700BF1D
:1055E800002C014030B4036A23F480730362036A19
:1055F8004468C26922F4803222F073020D682A439B
:1056080023F400738D6843EA0523184DA84203D09C
:1056180005F50065A84206D123F40063CD6843EA86
:10562800052323F48063114DA8420FD005F50065CA
:10563800A8420BD005F54065A84207D005F580655E
:10564800A84203D005F58065A84207D124F4405C40
:105658004C694CEA041C8C694CEA04144460C2612D
:105668004A68C263036230BC704700BF002C014027
:1056780030B4036A23F480530362036A4468C2693E
:1056880022F0807222F4E6420D6842EA052223F4F1
:1056980000538D6843EA0533174DA84203D005F53A
:1056A8000065A84206D123F40043CD6843EA0533D8
:1056B80023F48043104DA8420FD005F50065A84299
:1056C8000BD005F54065A84207D005F58065A842CE
:1056D80003D005F58065A84207D124F4404C4C69F5
:1056E8004CEA841C8C694CEA84144460C2614A68A0
:1056F8000264036230BC7047002C014030B4036A76
:1057080023F480330362036A4468026D22F4803212
:1057180022F070020D682A4323F400338D6843EAAF
:1057280005430F4DA8420FD005F50065A8420BD0E0
:1057380005F54065A84207D005F58065A84203D065
:1057480005F58065A84204D124F480344D6944EA03
:105758000524446002654A688264036230BC70476D
:10576800002C014030B4036A23F480130362036AF7
:105778004468026D22F0807222F4E0420D6842EA29
:10578800052223F400138D6843EA05530F4DA84200
:105798000FD005F50065A8420BD005F54065A84275
:1057A80007D005F58065A84203D005F58065A842B5
:1057B80004D124F480244D6944EA852444600265B8
:1057C8004A68C264036230BC704700BF002C0140C5
:1057D80010B4036A046A24F001040462846924F0A2
:1057E800F00C4CEA021223F00A030B4382610362B5
:1057F8005DF8044B704710B4046A24F01004046286
:105808008469036A24F4704C4CEA023223F0A00342
:1058180043EA0113826103625DF8044B70478368B1
:1058280023F4401323F070030B4343F00703836012
:10583800704770477047704770477047704710B59A
:10584800044603681A6912F0020F12D0DA6812F0DF
:10585800020F0ED06FF002021A610123037703686A
:105868009B6913F0030F00F09F80FFF7E5FF00230B
:10587800237723681A6912F0040F13D0DA6812F03C
:10588800040F0FD06FF004021A61022323772368F4
:105898009B6913F4407F00F08D802046FFF7CCFF12
:1058A8000023237723681A6912F0080F12D0DA68E8
:1058B80012F0080F0ED06FF008021A610423237744
:1058C8002368DB6913F0030F7BD02046FFF7B4FF92
:1058D8000023237723681A6912F0100F12D0DA68B0
:1058E80012F0100F0ED06FF010021A610823237700
:1058F8002368DB6913F4407F6AD02046FFF79CFFDA
:105908000023237723681A6912F0010F03D0DA689D
:1059180012F0010F63D123681A6912F0800F03D0C7
:10592800DA6812F0800F61D123681A6912F4807F57
:1059380003D0DA6812F0800F5FD123681A6912F079
:10594800400F03D0DA6812F0400F5DD123681A695E
:1059580012F0200F03D0DA6812F0200F5BD1236811
:105968001A6912F4801F03D0DA6812F4801F59D123
:1059780023681A6912F4001F03D0DA6812F4001FB2
:1059880057D123681A6912F4800F03D0DA6812F429
:10599800800F55D123681A6912F4000F03D0DA6812
:1059A80012F4000F53D110BDFFF745FF2046FFF753
:1059B80044FF5CE72046FFF73EFF2046FFF73DFF28
:1059C8006EE72046FFF737FF2046FFF736FF7FE7F1
:1059D8002046FFF730FF2046FFF72FFF90E76FF0D4
:1059E80001021A612046FFF725FF94E76FF0800255
:1059F8001A61204600F069FC96E76FF480721A611C
:105A0800204600F063FC98E76FF040021A612046D8
:105A1800FFF714FF9AE76FF020021A61204600F0A2
:105A280053FC9CE76FF480121A61204600F04FFC8B
:105A38009EE76FF400121A61204600F049FCA0E7C7
:105A48006FF480021A61204600F043FCA2E76FF46D
:105A580000021A61204600F03DFCA4E703682C4AC6
:105A680090420ED0B0F1804F0BD0A2F59432904204
:105A780007D002F58062904203D002F59632904238
:105A880003D123F070034A681343214A90421AD085
:105A9800B0F1804F17D0A2F59432904213D002F59E
:105AA800806290420FD002F5963290420BD002F5F8
:105AB8004062904207D002F58062904203D002F51E
:105AC8008062904203D123F44073CA68134323F0E1
:105AD80080034A69134303608B68C3620B6883625F
:105AE8000B4B98420FD003F5006398420BD003F597
:105AF8004063984207D003F58063984203D003F5CA
:105B08008063984201D10B690363012343617047A5
:105B1800002C014060B310B5044690F83D3013B333
:105B2800022384F83D30214651F8040BFFF796FF15
:105B3800012384F8483084F83E3084F83F3084F8F4
:105B4800403084F8413084F8423084F8433084F897
:105B5800443084F8453084F8463084F8473084F877
:105B68003D30002010BD80F83C30FBF725FED7E71C
:105B78000120704760B310B5044690F83D3013B368
:105B8800022384F83D30214651F8040BFFF766FFE5
:105B9800012384F8483084F83E3084F83F3084F894
:105BA800403084F8413084F8423084F8433084F837
:105BB800443084F8453084F8463084F8473084F817
:105BC8003D30002010BD80F83C30FFF732FED7E7AB
:105BD8000120704730B4036A23F010030362036A9C
:105BE8004468826922F0807222F4E6420D6842EA33
:105BF800052223F020038D6843EA0513174DA842B8
:105C080003D005F50065A84206D123F08003CD68CE
:105C180043EA051323F04003104DA8420FD005F5C1
:105C28000065A8420BD005F54065A84207D005F5E8
:105C38008065A84203D005F58065A84207D124F401
:105C4800406C4C694CEA840C8C694CEA84044460CE
:105C580082614A688263036230BC7047002C01404D
:105C680038B590F83C30012B00F0958004460D467D
:105C7800012380F83C30142A00F28880DFE802F023
:105C88000B8686861F86868634868686488686861E
:105C98005D86868671000068FFF754FC2268936968
:105CA80043F0080393612268936923F00403936126
:105CB8002268936929690B439361002067E00068B3
:105CC800FFF788FF2268936943F4006393612268B1
:105CD800936923F48063936122689369296943EA8D
:105CE80001239361002052E00068FFF77BFC2268E3
:105CF800D36943F00803D3612268D36923F004030E
:105D0800D3612268D36929690B43D36100203EE03F
:105D18000068FFF7ADFC2268D36943F40063D361E0
:105D28002268D36923F48063D3612268D36929691F
:105D380043EA0123D361002029E00068FFF7DEFC75
:105D48002268136D43F0080313652268136D23F06E
:105D5800040313652268136D29690B43136500203A
:105D680015E00068FFF7FEFC2268136D43F400633A
:105D780013652268136D23F4806313652268136D1D
:105D8800296943EA01231365002000E0012000236C
:105D980084F83C3038BD0220FCE710B4846824F451
:105DA8007F4C42EA03220A4342EA0C0282605DF811
:105DB800044B704790F83C30012B00F08F8010B5F1
:105DC8000446012380F83C30022380F83D30026805
:105DD8009068434B034093600B68702B55D031D8C3
:105DE800502B6CD00CD9602B2AD1CA68496820681E
:105DF800FFF701FD60212068FFF711FD002035E065
:105E0800402B0AD1CA6849682068FFF7E1FC4021A5
:105E18002068FFF704FD002028E05BD8202B07D07E
:105E280003D9302B04D0012020E00BB1102B05D171
:105E380019462068FFF7F3FC002017E0012015E061
:105E4800012013E0B3F5005F2CD00BD9254A93420B
:105E5800EED012D9244A9342EAD030329342E7D0A6
:105E6800012003E0B3F5805F36D10020012384F8D8
:105E78003D30002384F83C3010BDB3F1101FD7D05B
:105E8800103A9342D4D00120F0E7CB684A68896879
:105E98002068FFF782FF2268936843F077039360D6
:105EA8000020E3E7CB684A6889682068FFF775FF38
:105EB8002268936843F4804393600020D6E7CA6859
:105EC80049682068FFF784FC50212068FFF7A7FC89
:105ED8000020CBE70120C9E70120C7E7022070476F
:105EE8008800CEFF300010004000100001F01F01B4
:105EF800012303FA01FC036A23EA0C030362036A21
:105F080002FA01F10B4303627047000010B5044622
:105F18000846002947D194F83E30DBB2013B18BF50
:105F28000123002B40F09480002867D1022384F8D5
:105F38003E30012201462068FFF7D8FF2368474A10
:105F480093420FD002F5006293420BD002F54062F3
:105F5800934207D002F58062934203D002F5806233
:105F6800934203D15A6C42F400425A6423683B4A74
:105F780093425FD0B3F1804F5CD0A2F59432934244
:105F880058D002F58062934254D002F5963293427B
:105F980050D002F5406293424CD01A6842F0010298
:105FA8001A60002055E004290CD0082911D00C29CA
:105FB80016D010291BD094F84330DBB2013B18BF30
:105FC8000123AEE794F83F30DBB2013B18BF012351
:105FD800A7E794F84030DBB2013B18BF0123A0E7E4
:105FE80094F84130DBB2013B18BF012399E794F8DC
:105FF8004230DBB2013B18BF012392E7042809D0E5
:1060080008280BD00C280DD010280FD0022384F8B4
:1060180043308EE7022384F83F308AE7022384F86E
:10602800403086E7022384F8413082E7022384F86F
:1060380042307EE799680A4A0A40062A0AD0B2F531
:10604800803F09D01A6842F001021A60002000E07F
:10605800012010BD0020FCE70020FAE7002C0140D9
:106068000700010001F01F01042303FA01FC036A81
:1060780023EA0C030362036A02FA01F10B43036289
:106088007047000010B504460846002933D194F83B
:106098004430DBB2013B18BF0123002B62D100283A
:1060A80042D1022384F84430042201462068FFF7D5
:1060B800D9FF2268536C43F40043536423682C4A85
:1060C800934241D0B3F1804F3ED0A2F5943293422F
:1060D8003AD002F58062934236D002F59632934266
:1060E80032D002F5406293422ED01A6842F0010283
:1060F8001A60002037E0042908D008290DD094F848
:106108004730DBB2013B18BF0123C6E794F845309E
:10611800DBB2013B18BF0123BFE794F84630DBB27E
:10612800013B18BF0123B8E7042805D0082807D089
:10613800022384F84730B7E7022384F84530B3E7F1
:10614800022384F84630AFE799680A4A0A40062ACB
:106158000AD0B2F5803F09D01A6842F001021A60ED
:10616800002000E0012010BD0020FCE70020FAE735
:10617800002C01400700010090F83C30012B40D072
:1061880030B4012380F83C30022380F83D300268A7
:10619800536894681C4DAA4203D005F50065AA42CD
:1061A80003D123F470034D682B4323F0007323F0CD
:1061B80070030D682B4353600368134A934212D04F
:1061C800B3F1804F0FD0A2F5943293420BD002F571
:1061D8008062934207D002F59632934203D002F5CB
:1061E8004062934204D124F080048A6814439C607E
:1061F800012380F83D30002380F83C30184630BC3D
:1062080070470220704700BF002C014090F83C30D6
:10621800012B55D010B4012380F83C30CB6823F40F
:1062280040738A68134323F480634A68134323F452
:1062380000630A68134323F480530A69134323F461
:1062480000534A69134323F480430A6B134323F42E
:1062580070238A6943EA024302681A4CA24203D0B7
:1062680004F50064A24203D123F08053CC69234390
:10627800144CA2420BD004F50064A24207D0536428
:10628800002380F83C3018465DF8044B704723F42F
:1062980070038C6A43EA045323F080730C6A234327
:1062A80023F000734C6A2343064CA24203D004F542
:1062B8000064A242E3D123F00053C96A0B43DEE72E
:1062C80002207047002C01407047704770477047A4
:1062D80070477047704703460020A3F844004BF608
:1062E8008072A3F840207047B0F8403023F47E5302
:1062F8005B045B0CA0F840300020704784B08446F3
:1063080001A880E80E000123ACF840300020ACF86A
:106318004000ACF84400ACF8500004B0704710B529
:1063280003460A7830F822C01FFA8CFC2CF4EC4C97
:106338002CF0700C1FFA8CFCC878032862D8DFE8B0
:1063480000F0565D0259002048F2800E4CEA0E0C0F
:1063580023F822C091F800C033F82C2012B222F49E
:10636800E04222F070024CEA020292B242EA0E02C5
:1063780023F82C200A7B002A40F0C2804A78002AA1
:1063880051D0B3F8502013FA82F20C7802EBC40211
:10639800B1F806C04FEA5C0C4FEA4C0CA2F800C4F6
:1063A8000C7833F8242012F0400F0CD033F8242056
:1063B80092B222F4E04222F0700242F4004242F02B
:1063C800C00223F82420CA78012A1DD0097833F89E
:1063D800212092B222F4E04222F0400282F0200210
:1063E80042F4004242F0800223F8212066E04CF497
:1063F800007CA9E74CF4C06C0020A5E74CF4806C45
:106408000020A1E701209FE7097833F8212092B204
:1064180022F4E04222F0400242F4004242F08002BC
:1064280023F821204AE0B3F8502013FA82F20C78BE
:1064380002EBC402B1F806C04FEA5C0C4FEA4C0C00
:10644800A2F804C4B3F8502013FA82F20C7802EBD5
:10645800C4020C693E2C32D94FEA541C14F01F0FA9
:1064680001D10CF1FF3C6FEACC6C6FEA5C4C1FFA6F
:106478008CFCA2F806C40C7833F8242012F4804F60
:106488000CD033F8242092B222F4E04222F07002B9
:1064980042F4404242F0800223F82420097833F87D
:1064A800212092B222F4804222F0700282F44052FB
:1064B80042F4004242F0800223F8212010BD8CB93A
:1064C800B2F80644A4B224F4F844A4B2A2F80644EC
:1064D800B2F806446FEA44446FEA5444A4B2A2F8FE
:1064E8000644C8E74FEA540C14F0010F01D00CF130
:1064F800010C4FEA8C2C1FFA8CFCA2F806C4BAE7F0
:10650800CA78022A72D00C7833F8242092B222F486
:10651800E24222F0700242F4004242F0800223F884
:106528002420B3F8502013FA82F291F800C002EB4D
:10653800CC02B1F808C04FEA5C0C4FEA4C0CA2F848
:1065480000C4B3F8502013FA82F291F800C002EBAD
:10655800CC02B1F80AC04FEA5C0C4FEA4C0CA2F826
:1065680004C44A78002A50D10C7833F8242012F455
:10657800804F0CD033F8242092B222F4E04222F06B
:10658800700242F4404242F0800223F824200C7842
:1065980033F8242012F0400F0CD033F8242092B2A4
:1065A80022F4E04222F0700242F4004242F0C002BB
:1065B80023F8242091F800C033F82C2092B222F45A
:1065C800804222F0700282F4405248F28004224352
:1065D80023F82C20097833F8212092B222F4E042E3
:1065E80022F04002224323F8212067E70C7833F891
:1065F800242092B222F4E04222F0700242F40142D6
:1066080042F0800223F824208BE70C7833F824200A
:1066180012F4804F0CD033F8242092B222F4E042D6
:1066280022F0700242F4404242F0800223F8242013
:106638000C7833F8242012F0400F0CD033F82420C3
:1066480092B222F4E04222F0700242F4004242F098
:10665800C00223F82420CA78012A1ED00C7833F807
:10666800242092B222F4E04222F0400282F020027A
:1066780042F4004242F0800223F82420097833F8DB
:10668800212092B222F4804222F0700242F40042A9
:1066980042F0800223F8212010E70C7833F82420F8
:1066A80092B222F4E04222F0400242F4004242F068
:1066B800800223F82420E1E70B7B002B46D14B789E
:1066C80013B30A7830F8223013F0400F0CD030F8AA
:1066D80022309BB223F4E04323F0700343F40043D9
:1066E80043F0C00320F822300A7830F822309BB2F9
:1066F80023F4E04323F0400343F4004343F08003D2
:1067080020F82230002070470A7830F8223013F43D
:10671800804F0CD030F822309BB223F4E04323F0B2
:10672800700343F4404343F0800320F822300A7892
:1067380030F822309BB223F4804323F0700343F4F3
:10674800004343F0800320F82230DBE74B78002B2E
:106758004ED10A7830F8223013F4804F0CD030F83C
:1067680022309BB223F4E04323F0700343F4404308
:1067780043F0800320F822300A7830F8223013F0F2
:10678800400F0CD030F822309BB223F4E04323F0C2
:10679800700343F4004343F0C00320F822300A7822
:1067A80030F822309BB223F4E04323F0700343F423
:1067B800004343F0C00320F822300B7830F8232040
:1067C80092B222F4804222F0700248F2800C42EA2F
:1067D8000C0220F823200A7830F822309BB223F4E8
:1067E800E04323F0400343EA0C0320F8223089E712
:1067F8000A7830F8223013F4804F0CD030F8223069
:106808009BB223F4E04323F0700343F4404343F086
:10681800800320F822300A7830F8223013F0400F35
:106828000CD030F822309BB223F4E04323F07003FD
:1068380043F4004343F0C00320F822300A7830F8CC
:1068480022309BB223F4E04323F0700343F4404327
:1068580043F0800320F822300B7830F8232092B2DE
:1068680022F4E04222F0400248F2800C42EA0C0294
:1068780020F823200A7830F822309BB223F4804392
:1068880023F0700343EA0C0320F822303AE74B78F0
:106898008BB10A7830F822309BB223F4E04323F01E
:1068A800400383F0100343F4004343F0800320F8CF
:1068B8002230002070470A7830F822309BB223F447
:1068C800804323F0700383F4805343F4004343F080
:1068D800800320F82230ECE70B7B002B4BD14B7860
:1068E80033B30A7830F8223013F0400F0CD030F868
:1068F80022309BB223F4E04323F0700343F40043B7
:1069080043F0C00320F82230CB78012B33D00A782B
:1069180030F822309BB223F4E04323F0400383F0A5
:10692800200343F4004343F0800320F8223022E0A0
:106938000A7830F8223013F4804F0CD030F8223027
:106948009BB223F4E04323F0700343F4404343F045
:10695800800320F822300A7830F822309BB223F4E2
:10696800804323F0700383F4405343F4004343F01F
:10697800800320F822300020704711B98023A0F846
:106988004C3000207047B0F858306FEA43436FEA44
:1069980053439BB2A0F8583000207047B0F8440029
:1069A80080B2704710B45C1C6408024402F580622F
:1069B80007E00B78487843EA002322F8023B0231CB
:1069C800013C002CF5D15DF8044B704770B50546C5
:1069D8000C464A78012A32D00B7B002B40F0838288
:1069E8008B690A69934240F25D829B1A8B61B5F804
:1069F800503015FA83F3217803EBC1033E2A40F2A5
:106A08005582510912F01F0F00D101396FEAC16197
:106A18006FEA514189B2A3F80614227835F822307A
:106A28009BB223F4804323F0700383F4405343F470
:106A3800004343F0800325F82230002070BD8E69A2
:106A480009698E4200D90E46237B2BB3E378022BCB
:106A580044D0236A9B1B2362237835F8231011F056
:106A6800400F00F0DC81002A40F0C981B5F85020C1
:106A780015FA82F202EBC3033E2E40F2A38172099B
:106A880016F01F0F00D1013A6FEAC2626FEA524254
:106A980092B2A3F80624BBE1B6B23346E288616934
:106AA8002846FFF77FFFB5F8503015FA83F32278B0
:106AB80003EBC203A3F80264227835F822309BB2B4
:106AC80023F4E04323F0400383F0300343F400430E
:106AD80043F0800325F822300020AFE7236A99426B
:106AE80080F05281227835F822309BB223F4E043BB
:106AF80023F0700343F4014343F0800325F8223068
:106B0800236A9B1B2362237835F8232012F0400F59
:106B180000F09D8062788ABBB5F8502015FA82F2A1
:106B280002EBC3033E2E0CD9720916F01F0F00D1D9
:106B3800013A6FEAC2626FEA524292B2A3F806249F
:106B48001EE08EB9B3F8062492B222F4F84292B24B
:106B5800A3F80624B3F806246FEA42426FEA5242C9
:106B680092B2A3F806240BE0720816F0010F00D0C9
:106B78000132920292B2A3F8062401E0012A27D03A
:106B8800B3B2628961692846FFF70CFF6369334431
:106B98006361236A2269934224D99B1B2362637829
:106BA800002B40D1B5F8503015FA83F3227803EB67
:106BB800C2033E2E1AD9720916F01F0F00D1013AEE
:106BC8006FEAC2626FEA524292B2A3F802242CE042
:106BD800B5F8502015FA82F202EBC303B2B2A3F85B
:106BE8000624CDE7002222621E46D8E78EB9B3F804
:106BF800022492B222F4F84292B2A3F80224B3F823
:106C080002246FEA42426FEA524292B2A3F8022487
:106C18000BE0720816F0010F00D00132920292B216
:106C2800A3F8022401E0012B06D0B3B222896169DE
:106C38002846FFF7B7FE3FE7B5F8503015FA83F35B
:106C4800227803EBC203B2B2A3F80224EDE762781C
:106C58008ABBB5F8502015FA82F202EBC3033E2E28
:106C68000CD9720916F01F0F00D1013A6FEAC262FF
:106C78006FEA524292B2A3F802241EE08EB9B3F82A
:106C8800022492B222F4F84292B2A3F80224B3F892
:106C980002246FEA42426FEA524292B2A3F80224F7
:106CA8000BE0720816F0010F00D00132920292B286
:106CB800A3F8022401E0012A27D0B3B2228961692E
:106CC8002846FFF76FFE636933446361236A2269CC
:106CD800934224D99B1B23626378002B40D1B5F8DB
:106CE800503015FA83F3227803EBC2033E2E1AD9EB
:106CF800720916F01F0F00D1013A6FEAC2626FEAFB
:106D0800524292B2A3F806242CE0B5F8502015FAA6
:106D180082F202EBC303B2B2A3F80224CDE7002249
:106D280022621E46D8E78EB9B3F8062492B222F43E
:106D3800F84292B2A3F80624B3F806246FEA424256
:106D48006FEA524292B2A3F806240BE0720816F0DA
:106D5800010F00D00132920292B2A3F8062401E09A
:106D6800012B06D0B3B2628961692846FFF71AFE83
:106D7800A2E6B5F8503015FA83F3227803EBC20384
:106D8800B2B2A3F80624EDE7217835F8212092B2B3
:106D980022F4E24222F0700242F4004242F0800201
:106DA80025F82120B5F8502015FA82F2217802EB57
:106DB800C1029BB2A2F80234228961692846FFF712
:106DC800F1FD79E68EB9B3F8062492B222F4F842BE
:106DD80092B2A3F80624B3F806246FEA42426FEA97
:106DE800524292B2A3F8062412E0720816F0010F7C
:106DF80000D00132920292B2A3F8062408E0B5F856
:106E0800502015FA82F202EBC303B2B2A3F80624AB
:106E1800B3B2628961692846FFF7C4FD4CE68ABBB4
:106E2800B5F8502015FA82F202EBC3033E2E0CD9B6
:106E3800720916F01F0F00D1013A6FEAC2626FEAB9
:106E4800524292B2A3F8022425E08EB9B3F8022484
:106E580092B222F4F84292B2A3F80224B3F80224C0
:106E68006FEA42426FEA524292B2A3F8022412E059
:106E7800720816F0010F00D00132920292B2A3F804
:106E8800022408E0B5F8502015FA82F202EBC30399
:106E9800B2B2A3F80224B3B2228961692846FFF787
:106EA80081FD09E600228A611A46A0E58AB9B3F88D
:106EB800062492B222F4F84292B2A3F80624B3F858
:106EC80006246FEA42426FEA524292B2A3F80624BD
:106ED800A3E5510812F0010F00D00131890289B2EF
:106EE800A3F8061499E5CB78022B3BD0012B40F090
:106EF8001B8189692369994240F2CA80C91AA16134
:106F0800AAB9B5F8502015FA82F2217802EBC1022D
:106F18003E2B40F2C180590913F01F0F00D10139EF
:106F28006FEAC1616FEA514189B2A2F8021462782E
:106F3800002A40F0EB80B5F8502015FA82F221784B
:106F480002EBC1023E2B40F2C480590913F01F0F17
:106F580000D101396FEAC1636FEA53439BB2A2F8CB
:106F680006345AE5AAB9B0F8503010FA83F30A7813
:106F780003EBC20309693E2925D94A0911F01F0FFD
:106F880000D1013A6FEAC2626FEA524292B2A3F8A4
:106F980002246378002B50D1B5F8503015FA83F3EA
:106FA800227803EBC20321693E2929D94A0911F045
:106FB8001F0F00D1013A6FEAC2626FEA524292B2E1
:106FC800A3F806243BE089B9B3F8022492B222F46C
:106FD800F84292B2A3F80224B3F802246FEA4242BC
:106FE8006FEA524292B2A3F80224D2E74A0811F09B
:106FF800010F00D00132920292B2A3F80224C8E72E
:1070080089B9B3F8062492B222F4F84292B2A3F8EE
:107018000624B3F806246FEA42426FEA524292B25B
:10702800A3F806240BE04A0811F0010F00D0013242
:10703800920292B2A3F8062401E0012B1DD0E36965
:10704800002B3FF4EAAC227835F8221044F24003D2
:1070580003EA01008B4302D000287FF4DEAC35F848
:1070680022309BB223F4E04323F0700343F400433F
:1070780043F0C00325F82230CFE4B5F8503015FAB4
:1070880083F3227803EBC203228AA3F80624D6E707
:107098000023A3610B4633E78BB9B2F8021489B217
:1070A80021F4F84189B2A2F80214B2F802146FEA86
:1070B80041416FEA514189B2A2F8021437E75908F1
:1070C80013F0010F00D00131890289B2A2F802142D
:1070D8002DE78BB9B2F806349BB223F4F8439BB280
:1070E800A2F80634B2F806346FEA43436FEA534312
:1070F8009BB2A2F8063490E4590813F0010F00D0AF
:1071080001318B029BB2A2F8063486E4012A7FF48F
:1071180084ACB5F8502015FA82F2217802EBC1024E
:107128009BB2A2F8063478E4012087E410B45C0826
:10713800104400F5806007E030F8022B0A70C2F3B3
:1071480007224A700231013C002CF5D113F0010FDF
:1071580001D003880B705DF8044B704710B5D0F868
:10716800BC4284B1D0F8C0327BB194F80002FF2849
:107178000DD09B6894F8012221469847FF2384F894
:107188000032002010BD0320FCE70020FAE70020B1
:10719800F8E70000432303800048704748000020B8
:1071A80043230380004870478C000020432303805A
:1071B80000487047DC0000200A230380004870471D
:1071C800D000002038B5D0F8BC5275B1044601F0A3
:1071D800D3F8C5F80C02D4F8C032DB6805F50371A2
:1071E800D5F804029847002038BD0320FCE710B505
:1071F800D0F8C442D0F8BC3253B301EB810200EBA3
:10720800820292694AB101EB810C04EBCC04A46BB5
:10721800B2FBF4FC04FB1C2272B10022C3F8142256
:10722800D0F8C0221469ACB10A4603F50471D3F84A
:107238000802A047002010BD01EB810300EB830387
:1072480000249C612346224601F086F82046F2E796
:107258000320F0E70020EEE7F0B583B0D0F8BC6279
:1072680000238DF80730ADF80430002E6CD00746A7
:107278000C460B7813F060052AD0202D5ED1CA8801
:10728800F2B113F0800F0FD0D0F8C0329B683146AE
:1072980060789847E288072A28BF0722314638468F
:1072A80000F0EEFD00254CE04B7886F800328B7933
:1072B80086F80132CA88314600F0F7FD002540E023
:1072C800D0F8C0329B68002248789847002538E0FB
:1072D8004E780B2E2ED8DFE806F006342D2D2D2DF6
:1072E8002D2D2D2D152490F89C32DBB2032B03D0C5
:1072F80000F08CFA032524E0022201A900F0C0FD69
:1073080035461EE090F89C32DBB2032B03D000F028
:107318007DFA032515E001220DF1070100F0B0FD0B
:107328000FE090F89C32DBB2032B0AD000F06EFA23
:10733800032506E000F06AFA032502E000F066FA89
:107348000325284603B0F0BD0325FAE738B50446FF
:10735800812100F0CAFF002525870121204600F081
:10736800C4FFA4F878518221204600F0BEFFA4F89B
:107378004C50A4F84E50D4F8BC324BB1D4F8C032BB
:107388005B689847D4F8BC0201F024F8C4F8BC52F2
:10739800002038BD70B504464FF4077001F016F8A8
:1073A800B8B30646C4F8BC02237CBBBB4FF40073D9
:1073B80002228121204600F08DFF012525874FF408
:1073C800007302222946204600F084FFA4F8785171
:1073D8001023A4F84E30082303228221204600F00F
:1073E80079FF0123A4F84C30D4F8C0321B689847C1
:1073F8000023C6F81432C6F81832257C15BB4FF4A2
:107408000073D6F804220121204600F0ADFF28467B
:1074180070BD0023C4F8BC320225F8E740230222DD
:107428008121204600F056FF0125258740230222AE
:107438002946204600F04EFFA4F878511023A4F8FE
:107448004E30C8E74023D6F804220121204600F038
:107458008BFF0025DBE719B1C0F8C0120020704788
:1074680003207047D0F8BC322BB1C3F80812C3F818
:1074780010220020704703207047D0F8BC321BB19F
:10748800C3F804120020704703207047D0F8BC22CC
:10749800A2B108B5D2F814320BB1012008BD0123FE
:1074A800C2F81432D2F81032C362D2F81032D2F8CD
:1074B8000822812100F050FF0020EFE703207047E9
:1074C80010B5D0F8BC2292B1047C44B94FF40073D3
:1074D800D2F80422012100F047FF204610BD4023C6
:1074E800D2F80422012100F03FFF0024F5E703242D
:1074F800F3E798B108B503460020C3F8B802C3F80B
:10750800C002C3F8CC0209B1C3F8B412012183F850
:107518009C121A70184600F091FE08BD03207047AF
:1075280010B582B00023ADF8063061B10446C0F84A
:10753800B812CB6A4BB10DF106009847C4F8CC02DB
:10754800002002B010BD0320FBE70020F9E708B5D2
:1075580000F0B8FE08BD08B5D0F8B83213B11B6802
:10756800984708BD0320FCE708B5D0F8B8320BB13E
:107578005B689847002008BD38B5044600F2AA2584
:10758800284600F02FF90123C4F89432B4F8B03239
:10759800C4F8983294F8AA1201F01F03012B0DD0F9
:1075A800022B10D02BB101F08001204600F0A5FE7F
:1075B80003E02946204600F0E4FA38BD2946204673
:1075C80000F017FBF9E72946204600F046FBF4E7F0
:1075D80038B504460D4641BB1346D0F89422032A19
:1075E80001D0084638BDD0F85C11D0F8602191422E
:1075F80009D890F89C32DBB2032B0FD0204600F05C
:107608006BFC2846EEE7891AC0F85C118A4228BF4D
:107618000A46194600F058FC2846E3E7D0F8B83285
:107628001B69002BEAD09847E8E790F89C32DBB258
:10763800032B01D00020D5E7D0F8B8329B690BB1F5
:107648009847CFE70020CDE738B504460D46002916
:107658004AD11346D0F89422022A05D094F8A032D1
:10766800012B3CD0284638BDC269016A8A420ED82F
:107678008A4218D094F89C32DBB2032B27D08021A1
:10768800204600F03AFE204600F031FCE6E7521AA8
:10769800C261194600F001FC00231A46194620462B
:1076A80000F062FEDAE783699942E3D8D0F89822BD
:1076B8009342DFD20022114600F0EFFB0021C4F80C
:1076C80098120B460A46204600F04EFEC6E7D4F84C
:1076D800B832DB68002BD2D020469847CFE700238A
:1076E80084F8A0322846BEE790F89C32DBB2032B20
:1076F80001D00020B7E7D0F8B8325B690BB19847E2
:10770800B1E70020AFE7012380F89C320023C0F8DE
:1077180094324360C0F8A432D0F8B832F3B170B5EF
:107728000446D0F8BC221AB15B680BB10021984717
:10773800402300221146204600F0CCFD0126A4F883
:1077480064614025C4F860512B4600228021204600
:1077580000F0C0FDA6842562002070BD032070479C
:1077680001740020704790F89C32DBB280F89D329B
:10777800042380F89C320020704790F89C32DBB2DA
:10778800042B01D00020704790F89D32DBB280F8BE
:107798009C32F7E7D0F8B82262B108B590F89C326D
:1077A800DBB2032B01D0002008BDD36923B1984771
:1077B8000020F9E7032070470020F5E70346002082
:1077C80002E00130C0B201331A78002AF9D17047BB
:1077D80008B54B88012B00D008BDC0F8A43200F0D2
:1077E8007BFBF9E70B7803704B7843708B78CA788A
:1077F80043EA022343800B794A7943EA02238380D0
:107808008B79CA7943EA0223C380704710B50446CE
:10781800802100F072FD0021204600F06EFD10BDB1
:1078280030B583B004460D460023ADF806304A88CB
:10783800130A013B0E2B00F2BC80DFE803F0153081
:1078480044BABA9EABBABABABABABABA0800D0F849
:10785800B432DB6923B10DF10601007C98470AE0D8
:107868002946FFF7D3FF18E0D0F8B4321B680DF1B2
:107878000601007C9847EA88002A00F0A380BDF83A
:107888000630002B00F099809A4228BF1A46ADF8BE
:1078980006200146204600F0F3FA03B030BD037C11
:1078A80043B9D0F8B8329B6A0DF106009847022315
:1078B8004370E0E7D0F8B832DB6A0DF1060098476C
:1078C80002234370D7E7D2B2052A52D8DFE802F084
:1078D80003101D2A3744D0F8B4325B6823B10DF188
:1078E8000601007C9847C6E72946FFF78FFFD4E7D3
:1078F800D0F8B4329B6823B10DF10601007C98479B
:10790800B9E72946FFF782FFC7E7D0F8B432DB684A
:1079180023B10DF10601007C9847ACE72946FFF733
:1079280075FFBAE7D0F8B4321B6923B10DF106012F
:10793800007C98479FE72946FFF768FFADE7D0F836
:10794800B4325B6923B10DF10601007C984792E7D8
:107958002946FFF75BFFA0E7D0F8B4329B6923B153
:107968000DF10601007C984785E72946FFF74EFF91
:1079780093E72946FFF74AFF8FE7037C33B9D0F82E
:10798800B8325B6B0DF10600984774E72946FFF79C
:107998003DFF82E7037C43B9D0F8B8321B6B0DF189
:1079A800060098470723437065E72946FFF72EFF2F
:1079B80073E72946FFF72AFF6FE729462046FFF7B6
:1079C80025FF6AE7204600F087FA66E738B50446DF
:1079D8008B88FBB9CB88EBB94B887F2B1AD803F07F
:1079E8007F0590F89C32DBB2032B0CD080F89E52B6
:1079F800294600F0A9FC204600F06EFA35B10223B2
:107A080084F89C3209E0FFF701FF06E0012384F8BF
:107A18009C3202E02046FFF7F9FE38BD70B50446F7
:107A28000E468D782E4B1D70012D10D890F89C3283
:107A3800DBB2022B0FD0032B23D0FFF7E7FE284B36
:107A480019782046FFF790FD0325284670BDFFF7FB
:107A5800DDFE0325F9E78DB145602946FFF77BFD7B
:107A6800054620B131462046FFF7D0FEEDE7204617
:107A780000F032FA032384F89C32E6E700F02CFA8F
:107A8800E3E7CDB141688D4225D0C9B2FFF76CFD5F
:107A9800134B197861602046FFF75DFD0546B0B1CC
:107AA80031462046FFF7B2FE21792046FFF75CFDFC
:107AB800022384F89C32C8E7022380F89C32456090
:107AC8002946FFF751FD204600F006FABDE720469B
:107AD80000F002FAB9E700F0FFF90025B5E700BFAA
:107AE800E80E002008B5CB88012B0BD190F89C320A
:107AF800DBB2022B09D9032B09D10122011D00F0A9
:107B0800BFF901E0FFF782FE08BD5BB213B9FFF7CA
:107B18007DFEF9E70146002341F8083F012200F005
:107B2800AFF9F1E708B590F89C32013B022B12D867
:107B3800CB88022B0CD10123C360D0F8A4320BB13F
:107B48000323C360022200F10C0100F099F908BD7B
:107B5800FFF75CFEFBE7FFF759FEF8E708B590F87A
:107B68009C32013B022B09D84B88012B00D008BD61
:107B78000023C0F8A43200F0AFF9F8E7FFF746FE9B
:107B8800F5E738B50C7804F06004202C06D0402CBA
:107B980004D054B1FFF73AFE002404E0D0F8B8321C
:107BA8009B6898470446204638BD4D78092D1DD856
:107BB800DFE805F012191C161C08051C0F0BFFF74F
:107BC8002FFEF0E7FFF702FFEDE7FFF727FF044678
:107BD800E9E7FFF787FFE6E7FFF7A4FF2C46E2E7B0
:107BE800FFF7F6FDDFE7FFF7B9FFDCE7FFF70EFE6B
:107BF800D9E770B505460C460B7803F06003202BD7
:107C080007D0402B05D023B1FFF700FE00263046F1
:107C180070BD95F89C32013B022B18D82379012BB3
:107C28000FD8D5F8B8329B682146284698470646AB
:107C3800E388002BEBD10028E9D1284600F04CF965
:107C4800E5E721462846FFF7E1FD0026DFE7214664
:107C58002846FFF7DBFD0026D9E7F8B506460D46AE
:107C68008B880C7804F06004202C08D0D9B2402C02
:107C780005D06CB12946FFF7C9FD002406E0D6F807
:107C8800B8329B6829463046984704462046F8BDD6
:107C98006F78012F2FD0032F05D0002F59D02946F8
:107CA800FFF7B4FDF2E790F89C32DBB2022B05D067
:107CB800032B12D02946FFF7A9FDE7E709B1802970
:107CC80004D129463046FFF7A1FDDFE700F015FB98
:107CD8008021304600F011FBD8E76B8823B919B131
:107CE800802901D0EB881BB1304600F0F5F8CDE7CC
:107CF80000F003FBF8E790F89C32DBB2022B05D0CA
:107D0800032B12D02946FFF781FDBFE709B180296F
:107D180004D129463046FFF779FDB7E700F0EDFAC0
:107D28008021304600F0E9FAB0E76B88002BADD12E
:107D380011F07F0F0AD1304600F0CEF8D6F8B832ED
:107D48009B6829463046984704469FE700F0DDFACD
:107D5800F1E790F89C22D2B2022A06D0032A29D051
:107D68002946FFF753FD3C4690E709B1802913D116
:107D780013F0800F15D101F07F0101EB810189001B
:107D880001F5A8713144043100230B60022230460A
:107D980000F076F83C4679E72946FFF737FD3C4680
:107DA80074E701F07F0101EB810189001031314452
:107DB8000431E9E75BB2002B1FDB01F00F0202EB95
:107DC800820200EB8202B2F8642122B3002B27DB87
:107DD80001F07F0303EB83039C0004F5A87434448B
:107DE800043409B1802924D10023236002222146CA
:107DF800304600F045F83C4648E701F00F0202EB38
:107E0800820200EB8202928C002ADFD12946FFF71A
:107E1800FDFC3C463AE72946FFF7F8FC3C4635E7C7
:107E280001F07F0303EB83039C00103434440434D3
:107E3800D7E7304600F071FA10B101232360D5E787
:107E480000232360D2E7D0B170B50D46164604462C
:107E5800FFF7B4FC431C5B009BB233802B700323F9
:107E68006B70022307E0EA5401345A1CD2B2002195
:107E7800A9540233DBB22278002AF4D170BD7047CE
:107E880008B513460222C0F894228361C3610A46EA
:107E9800002100F061FA002008BD08B513460A4623
:107EA800002100F059FA002008BD08B51346032246
:107EB800C0F89422C0F85831C0F85C310A46002155
:107EC80000F052FA002008BD08B513460A46002102
:107ED80000F04AFA002008BD08B50422C0F8942230
:107EE80000231A46194600F037FA002008BD08B5E5
:107EF8000522C0F8942200231A46194600F034FAE5
:107F0800002008BD08B500220F491048FFF7F1FA14
:107F180070B90F490D48FFF703FB60B90D490B48CD
:107F2800FFF799FA50B90948FFF711FB48B908BD9E
:107F3800F9F76EFAEDE7F9F76BFAEFE7F9F768FA90
:107F4800F1E7F9F765FAF2E734010020EC0E0020BA
:107F580010000020200100200020704700207047FA
:107F68000020704710B50146044C2046FFF785FAFB
:107F78002046FFF7A5FA002010BD00BFEC0E002038
:107F880010B5064C002206492046FFF76BFA054952
:107F98002046FFF772FA002010BD00BFEC0E00204B
:107FA800BC150020BC110020094BD3F8BC32D3F813
:107FB80014320BB10120704710B5054C0A46014632
:107FC8002046FFF74FFA2046FFF760FA10BD00BFC2
:107FD800EC0E002012230B8000487047540100204B
:107FE80004230B8000487047680100200023934257
:107FF8001ED200B510E00CF1370C01F813C00001D7
:108008004FEA430C0CF1010C4FF0000E01F80CE0A4
:108018000133DBB2934209D24FEA107CB0F1204F12
:10802800E9D20CF1300C01F813C0E8E75DF804FB65
:108038007047000038B50B4BD3F89005D3F894453A
:10804800D3F89835C01800D138BD074D0822A91CAF
:10805800FFF7CCFF042205F112012046FFF7C6FF07
:10806800F2E700BF0070FF1F6C01002008B51A235B
:108078000B80FFF7DFFF014808BD00BF6C0100203F
:1080880008B50A4628B905490548FFF7DCFE034844
:1080980008BD02490248FFF7D6FEF8E7BC190020E0
:1080A8003492000810B50A46034C21460348FFF7EE
:1080B800CAFE204610BD00BFBC1900204C92000823
:1080C80008B50A4628B905490548FFF7BCFE034824
:1080D80008BD02490248FFF7B6FEF8E7BC190020C0
:1080E8006092000808B50A4628B905490548FFF70F
:1080F800AAFE034808BD02490248FFF7A4FEF8E7B4
:10810800BC1900206C920008032805D8DFE800F0AD
:1081180005040205012070470320704708B5F9F7E8
:1081280079F908BD10B592B004464422002101A88F
:1081380000F076F92268114B9A4201D012B010BDB6
:108148004FF40053019301A8FDF716F890B90C4BB2
:108158009A6D42F400029A659B6D03F40003009344
:10816800009B002211461420FAF762FF1420FAF748
:1081780097FFE3E7F9F74CF9E9E700BF005C004037
:108188000010024008B500F52C71D0F8F002FFF796
:10819800F3F908BD08B501EB810300EBC303D3F87D
:1081A8007C21D0F8F002FFF713FA08BD08B501EBFF
:1081B800810300EBC303DA6BD0F8F002FFF744FA4F
:1081C80008BD08B5D0F8F002FFF7E4FA08BD10B50D
:1081D80004468368022B09D10121D4F8F002FFF785
:1081E800BFFAD4F8F002FFF78EFA10BDF9F710F9CC
:1081F800F2E7000010B50446D0F8F002FFF7B3FA32
:10820800A36923B1024A136943F00603136110BD41
:1082180000ED00E010B50446836923B9D4F8F002F4
:10822800FFF7ABFA10BD044A136923F00603136184
:10823800FFF774FFF2E700BF00ED00E010B5044659
:108248001E48C0F8F042C4F8C4021D4B036008235E
:108258004360022383600361002343618361C36138
:108268000362FBF794FB30BB182300221146D4F8B5
:10827800C402FCF7C6FA582300228021D4F8C402AD
:10828800FCF7BFFAC02300228121D4F8C402FCF70E
:10829800B8FA4FF4887300220121D4F8C402FCF71D
:1082A800B0FA4FF4807300228221D4F8C402FCF79C
:1082B800A8FA002010BDF9F7ABF8D5E7BC1B0020E1
:1082C800005C004008B5D0F8C402FBF7D2FBFFF70A
:1082D8001BFF08BD08B594461A466346D0F8C40289
:1082E800FCF758F9FFF710FF08BD08B5D0F8C4022D
:1082F800FCF792F9FFF708FF08BD08B5D0F8C402EB
:10830800FCF70FFAFFF700FF08BD08B5D0F8C40264
:10831800FCF73CFAFFF7F8FE08BDD0F8C43211F0BC
:10832800800F08D101F07F0101EB810103EBC1014E
:1083380091F86A01704701F07F01013101EB810179
:1083480003EBC1018878704708B5D0F8C402FCF780
:1083580034F8FFF7D9FE08BD08B5D0F8C402FCF719
:10836800B8F9FFF7D1FE08BD08B5D0F8C402FCF78C
:1083780085F9FFF7C9FE08BD08B5D0F8C402FCF7B7
:108388009FF908BD10B5044611B101290FD010BDE1
:10839800836923B9D4F8F002FFF7EFF9F7E7FFF79D
:1083A800BDFE094A136923F006031361F2E7D0F80A
:1083B800F002FFF7D8F9A369002BE8D0024A136945
:1083C80043F006031361E2E700ED00E00048704760
:1083D800B01E00207047000070B50D4E0D4D761B85
:1083E800B61006D0002455F8043B01349847A6423D
:1083F800F9D1094E094D761B00F004FFB61006D0DE
:10840800002455F8043B01349847A642F9D170BDC1
:108418005096000850960008589600085096000894
:10842800830730B548D0541E002A3FD0CAB203464D
:1084380001E0013C3AD303F8012B9D07F9D1032C45
:108448002DD9CDB245EA05250F2C45EA054536D983
:10845800A4F1100222F00F0C03F1200EE6444FEABB
:10846800121C03F1100242E9045542E90255103288
:108478007245F8D10CF1010214F00C0F03EB021253
:1084880004F00F0C13D0ACF1040323F003030433FE
:10849800134442F8045B9342FBD10CF003042CB163
:1084A800CAB21C4403F8012B9C42FBD130BD644680
:1084B8001346002CF4D1F9E703461446BFE71A46E1
:1084C800A446E0E7024B13B1024800F005B8704734
:1084D80000000000ED840008002301461A461846F3
:1084E80000F01AB838B5084B084D5B1B9C1007D034
:1084F800043B1D44013C55F804399847002CF9D138
:10850800BDE8384000F084BE5C9600085896000824
:10851800704700BF704700BF2DE9F047DFF880A023
:108528000646DAF8000098460F469146FFF7F0FF36
:108538001A4B1B68D3F8484124B365681F2D26DC05
:108548005EB96B1C0235DAF80000636044F82570E8
:10855800FFF7E0FF0020BDE8F08704EB8501012369
:10856800C1F88890D4F88821AB401A43022EC4F889
:108578008821C1F80881E4D1D4F88C211343C4F8C8
:108588008C31DEE703F5A674C3F84841D5E7DAF87D
:108598000000FFF7BFFF4FF0FF30DCE77C920008D8
:1085A800B005002010EE103A194A23F00043934218
:1085B8001CDDB3F1FF4F02DB30EE400A704700B517
:1085C80083B0684600F028F800F003000128DDEDCC
:1085D800010A9DED000A0ED0022813D070B100F0F8
:1085E8004DF9B1EE400A03B05DF804FBDFED090A6E
:1085F800002000F0FFBC00F041F9F4E7012000F092
:10860800F9FCF0E7012000F0F5FCB1EE400AEAE7DA
:10861800D80F493F0000000070B510EE103A894AA3
:1086280023F00044944286B0054670DD864A9442A1
:1086380010EE106A22DC002BDFED847A844A24F0E5
:108648000F04B0EE407A40F3E480944270EE677A0B
:1086580009BFDFED806A9FED807A9FED807A77EE23
:10866800E67A012077EEC76A77EEE67AC5ED006A0A
:1086780077EEC77AC5ED017A06B070BD784A9442A4
:1086880054DDB4F1FF4F49DAE215863AA4EBC25340
:1086980007EE903ABDEEE77ADFED726AB8EEC77A78
:1086A80077EEC77A8DED037A67EEA67ABDEEE77AA4
:1086B800B8EEC77A77EEC77A8DED047A67EEA67AB8
:1086C800F5EE407AF1EE10FACDED057A40F09080A3
:1086D800B5EE407AF1EE10FA14BF02230123624985
:1086E80001910221009103A8294600F049F9002EC2
:1086F800C2DA95ED007AD5ED017AB1EE477AF1EE5E
:10870800677A85ED007AC5ED017A4042B4E7002228
:1087180085ED000A4260002006B070BD70EE407A18
:108728000020C5ED017AC5ED007AA5E700F0AAFCA6
:108738009FED4E7A9FED456AF6EE007AE0EE077AF5
:108748009FED457AFDEEE77A17EE900AF8EEE76AB4
:108758001F28A6EEC60A66EE877AB1EE666A1EDCA8
:10876800434A411E24F0FF0352F82120934216D0B9
:1087780030EE677A85ED007A30EE470A002E30EE4B
:10878800670A85ED010ABFF677AFB1EE477AB1EE19
:10879800400A85ED007A85ED010A40426CE730EE2B
:1087A800677AE21517EE103AC3F3C753C3EBD454F4
:1087B800082CDFDDDFED277A9FED287AF0EE405AAE
:1087C800E6EE275A30EE650AA6EE270AF0EE407A62
:1087D800D6EE877A35EEE77A17EE103AC3F3C75329
:1087E800D21A192A06DCB0EE650A85ED007AC3E7CD
:1087F800032374E79FED1F7A9FED1F5AB0EE650AB9
:10880800A6EE070A75EEC07AE6EE077AD6EE857A06
:10881800AEE7944270EE277A09BFDFED0E6A9FED4E
:108828000E7A9FED0E7A77EEA67A4FF0FF3077EE4C
:10883800876A77EEE67AC5ED006A77EE877AC5ED46
:10884800017A19E7D80F493FE3CB1640800FC93F9B
:10885800D00FC93F004435374344353708A3852E28
:10886800800F4943000080430093000884F9223FA9
:108878008092000800A3852E32318D2410EE103A24
:1088880023F00043B3F1485F2CDAFDEEC07A17EE0F
:10889800903A002B60D020EE007ADFED317A9FED20
:1088A800315ADFED315A9FED316ADFED316AA7EEBB
:1088B800275ADFED307AE7EE055AA7EE256AE7EE8C
:1088C800067AE7EE276A67EE266A60EEC00AF6EED9
:1088D800007AE7EE260AB7EE000AD7EE270A30EE4E
:1088E800600A704720EE007ADFED1D7A9FED1D5A71
:1088F800DFED1D5A9FED1D6ADFED1D6A1E4AA7EECA
:10890800275A9342DFED1B7AE5EE075AA5EE876AF0
:10891800E6EE077AE7EE876A66EE876AD5DD174ADC
:10892800934214DC03F17F4307EE903AB7EE006AF6
:1089380036EE676A60EEC00AF6EE005AD7EE257A80
:10894800E7EE260A77EEE00A36EE600A7047B6EEE2
:10895800076AF5EE027AEDE7B7EE000A704700BF46
:108968004ED747ADF6740F317CF293B4010DD03772
:10897800ABAA2A3D610BB6BA9999993E0000483FC7
:108988002DE9F04F2DED048BDBB01C4603930691C7
:10899800A24B6899089253F82150111D824604F1A0
:1089A800FF38C0F2A382D31E48BF131DDB10029309
:1089B8000133DB000793DDE907239B1A0593029B2C
:1089C80015EB0801A3EB080316D401319FED947A47
:1089D800699819441EAA002BA4BF50F8234007EE3B
:1089E800904A03F10103ACBFF8EEE77AF0EE477A5C
:1089F8008B42E2EC017AEED1002DC0F2E782039BB4
:108A08001EAA02EB830446AE4FEA830C4046EF18D9
:108A18000AEB8301B8F1000FDFED817A09DB22460A
:108A28005346F3EC016A32ED017A8B42E6EE877A1F
:108A3800F7D10130B842E6EC017A04F10404E9D137
:108A480009AB0AAF03EB850907EB8503083B9FEDEC
:108A5800769ADFED748A059804930AEB0C0446AE07
:108A680000955AAB03EB8503002D13ED140A4FEA6A
:108A7800850B16DD06EB85033A4660EE097AB0EE03
:108A8800407AFDEEE77A73ED016AF8EEE77AB342D1
:108A9800A7EEE87A37EEA60ABDEEC77AA2EC017A0D
:108AA800EBD1019000F03CFBB0EE408AB4EE000A36
:108AB80028EE000A00F0EEFAF2EE007AA0EE678ADD
:108AC80001980028FDEEC89AF8EEE97A38EE678A30
:108AD80079DD05F1FF3EC0F1080357F82E1041FA81
:108AE80003FC0CFA03F3CB1AC0F1070219EE901A33
:108AF80043FA02F26144002A47F82E3009EE901A30
:108B080069DCB5EE408AF1EE10FA40F0C080009BB7
:108B180005F1FF3B5B4510DC05F18043013B07EBAA
:108B280083030021944653F804294B4541EA020186
:108B3800F9D16246002940F0F280009B013B57F8CA
:108B48002330002B40F0E780049B4FF0010C53F8D2
:108B580004290CF1010C002AF9D06B1CAC449E4688
:108B6800039A5119029A02EB030B0BF1804B699A95
:108B78000BF1FF3B06EB83051EAB02EB8B0B03EB04
:108B88008101DBED017A9FED267AF8EEE77AB8F1FC
:108B9800000F0BF1040BC1ED007A0A4601F1040144
:108BA80009DB534601E072ED017AF3EC016AA34256
:108BB800A6EEA77AF7D10EF1010EE645A5EC017AEB
:108BC800DFDD65464DE740F09C806B1E57F823209B
:108BD800D211002A95DD19EE903A002D03F1010318
:108BE80009EE903A40F39881396800297FD1012D28
:108BF80026D03B464FF0010C53F8041F00297AD0C9
:108C08000CF10103C1F580719D4247F82C1016DD67
:108C180057F82310BB4407EB83030AE04496000887
:108C280000000000000080430000803B0000C93FB6
:108C38001968C1F1FF0143F8041B5B45F8D1012114
:108C480000280CDD012800F04881022807D105F131
:108C5800FF3C57F82C3003F03F0347F82C30022A2A
:108C68007FF44FAFB7EE000A30EE488A00293FF490
:108C780048AF0992019000F053FA38EE408A099AF9
:108C88000198B5EE408AF1EE10FA3FF440AF029237
:108C9800DDE90732B0EE480A981A0195009D00F008
:108CA8003FFA1FED207AB4EEC70AF1EE10FADDE9BB
:108CB8000132C0F259815FED247A059960EE277A76
:108CC8000831FDEEE77A0591F8EEE77A03F1010B3A
:108CD800A7EEC70AFDEEE77ABDEEC00A10EE101A3D
:108CE80047F8231017EE903A47F82B302EE001236F
:108CF8004FF0000C86E70CF1010CAC457FF47CAF1B
:108D08009EE7F6EE007AB4EEE78AF1EE10FA80F20A
:108D1800F2800022F5E66B1C9E469C4620E70599EA
:108D2800A1F1080057F82B1005902B46009D69B952
:108D380003F18043023B07EB8303014653F8040920
:108D48000BF1FF3B08390028F8D0059105980092EF
:108D5800B7EE000A00F0E4F9BBF1000F009AC0F288
:108D680028814FEA8B0E46AB03EB0E060EF1040C7E
:108D78001FED537A07EB0C03311D73ED017AF8EE02
:108D8800E77ABB4267EE807A20EE070A61ED017A46
:108D9800F3D1002D1FED5B6A4FF0000420DB9348F0
:108DA800DFED937AB0EE467A3146002303E09C4229
:108DB80008DBB0EC017AF1EC016A01339D42E6EE82
:108DC800877AF4DA5AAB03EB8403A34543ED287A98
:108DD800A6F1040604F1010305D0002D1C46DEDAD5
:108DE800DFED837AEEE7689902291CDC002900F39D
:108DF80095800FD132ABDFED7E7A9C443CED017A51
:108E0800634577EE877AF9D10AB1F1EE677A069B66
:108E1800C3ED007A19EE903A03F007005BB0BDECA1
:108E2800048BBDE8F08F689B032BF3D1BBF1000FD7
:108E380000F0D4800EF5B4736B4432A913ED287A90
:108E480001EB8B0373ED017AF0EE476A37EE277A70
:108E5800994277EEC77A83ED007A77EEA67AC3ED6A
:108E6800017AEFD1BBF1010F40F3B8800BF1804BD1
:108E78000EF5B4730BF1FF3B0DEB030E4FEA8B0BB2
:108E88000BF104031EED287A0B4433A873ED017A25
:108E9800F0EE476A37EE277A984277EEC77A83ED85
:108EA800007A77EEA67AC3ED017AEFD10BF1080BC1
:108EB800DFED4F7A01EB0B03083133ED017A99426C
:108EC80077EE877AF9D1002A56D10699329A339BE0
:108ED8000A604B60C1ED027A9CE705F1FF3C57F848
:108EE8002C3003F07F0347F82C30B8E608230793AB
:108EF800002302935FE519EE903A002D03F1010378
:108F080009EE903AC8BF02223FF76EAEF7EE007A3C
:108F180037EEC88A0222F4E5002191E632A9DFED96
:108F2800347A01EB830333ED017A994277EE877A3D
:108F3800F9D19DED327A8ABB069BBBF1000FC3EDD8
:108F4800007A77EE677A0BDD33A90123B1EC017A59
:108F580001339B4577EE877AF8DA0AB1F1EE677A42
:108F6800069BC3ED017A55E7BDEEC00A9B4610EE9D
:108F7800101A47F82310E9E6DDED326A9DED337AE1
:108F8800069BF1EE666AB1EE477AF1EE677AC3EDB9
:108F9800006A83ED017AC3ED027A3BE7069BF1EEA6
:108FA800676ABBF1000F77EE677AC3ED006ACBDC26
:108FB800D4E7689B022B0DDC002B14DC7FF42AAF6E
:108FC800DFED0B7A002A3FF422AF1EE7039B4FEA3E
:108FD800830C35E5689B032B7FF41CAFDFED047A27
:108FE800002AC9D171E7DFED027AA2E71C960008D2
:108FF8000000000010EE103A23F00043B3F1485F80
:1090080004DAFDEEC07A17EE903A5BB360EE007AB0
:109018009FED157ADFED155A9FED156ADFED156A9C
:10902800E7EE875A9FED147AA5EEA76A20EE275A35
:10903800E6EE276AA6EEA77A30B9DFED106AE7EE0A
:10904800876AA6EE850A704727EE457AF6EE006A2B
:10905800A0EEA67ADFED0A6AD7EE270AE5EE260A21
:1090680030EE600A704700BFD3C92E2F342FD7B215
:109078001BEF3836010D50B98988083CABAA2ABEC7
:10908800ABAA2A3E10EE103A23F0004300EE103A45
:10909800704700BF10EE102AC2F3C7537F3B162B50
:1090A80022F0004128DC002B18DB1A4919410A423A
:1090B80021D0DFED197A70EE277AF5EEC07AF1EE5D
:1090C80010FA18DD002A04DA4FF4000040FA03F31E
:1090D8001A4422EA010300EE103A7047DFED0E7AD7
:1090E80070EE277AF5EEC07AF1EE10FA03DD002A69
:1090F80008DB9FED0A0A7047B1F1FF4FFBD330EE52
:10910800000A7047FFEE007A002918BFB0EE670A20
:10911800704700BFFFFF7F00CAF2497100000000DE
:1091280082B08DED010A019B33F000422AD0B2F1E2
:10913800FF4F23D213F0FF4F28D19DED017ADFEDC9
:109148002A7A2A4B67EE277A9842CDED017A37DBE7
:10915800019BC3F3C752193A0244FE2A1ADD9FED58
:10916800240A9FED247A019B002BF0EE407AB8BFC9
:10917800B0EE470A20EE270A02B0704730EE000A28
:1091880002B070479DED010A02B07047D20D02444B
:10919800FE2AE4DC002A0BDC12F1160F17DA4CF277
:1091A80050339842DBDC9FED140A9FED147ADAE71E
:1091B80023F0FF4343EAC25300EE103A02B070476F
:1091C8009FED0D0ADDED017A27EE800AD8E7193206
:1091D80023F0FF4343EAC253DFED097A07EE103A62
:1091E80027EE270ACCE700BF0000004CB03CFFFF89
:1091F800CAF24971CAF249F16042A20D6042A28DD9
:1092080000000033F8B500BFF8BC08BC9E467047A4
:0C921800F8B500BFF8BC08BC9E467047CB
:109224000000000000000000010203040607080912
:1092340053544D3332205669727475616C20436FF8
:109244006D506F727400000053544D6963726F6502
:109254006C656374726F6E696373000043444320EA
:10926400436F6E666967000043444320496E74652A
:10927400726661636500000088010020000FC93F29
:10928400000F494000CB9640000FC9400053FB40FB
:1092940000CB164100ED2F41000F494100316241DE
:1092A40000537B41003A8A4100CB9641005CA341C4
:1092B40000EDAF41007EBC41000FC94100A0D54183
:1092C4000031E24100C2EE410053FB4100F203428F
:1092D400003A0A420083104200CB164200141D4299
:1092E400005C234200A5294200ED2F42003636429D
:1092F400007E3C4200C74242000F4942A2000000E7
:10930400F9000000830000006E0000004E00000021
:10931400440000001500000029000000FC000000CB
:109324002700000057000000D1000000F5000000F5
:1093340034000000DD000000C0000000DB0000007D
:109344006200000095000000990000003C0000004D
:10935400430000009000000041000000FE000000F7
:109364005100000063000000AB000000DE000000BC
:10937400BB000000C500000061000000B700000051
:10938400240000006E0000003A00000042000000CB
:109394004D000000D2000000E000000006000000C4
:1093A400490000002E000000EA000000090000004F
:1093B400D1000000920000001C000000FE0000002C
:1093C4001D000000EB0000001C000000B1000000C4
:1093D40029000000A70000003E000000E800000093
:1093E4008200000035000000F50000002E0000009F
:1093F400BB0000004400000084000000E9000000FD
:109404009C0000007000000026000000B400000072
:109414005F0000007E0000004100000039000000F1
:1094240091000000D6000000390000008300000015
:109434005300000039000000F40000009C0000000C
:10944400840000005F0000008B000000BD000000ED
:10945400F9000000280000003B0000001F0000008D
:10946400F800000097000000FF000000DE0000008C
:1094740005000000980000000F000000EF0000004D
:109484002F000000110000008B0000005A000000B3
:109494000A0000006D0000001F0000006D000000C5
:1094A400360000007E000000CF000000270000000E
:1094B400CB00000009000000B70000004F000000CE
:1094C400460000003F000000660000009E0000000F
:1094D4005F000000EA0000002D000000750000009D
:1094E40027000000BA000000C7000000EB000000E5
:1094F400E5000000F10000007B0000003D000000DA
:109504000700000039000000F70000008A00000096
:109514005200000092000000EA0000006B0000000E
:10952400FB0000005F000000B10000001F0000000D
:109534008D0000005D0000000800000056000000DF
:10954400030000003000000046000000FC000000A2
:109554007B0000006B000000AB000000F000000086
:10956400CF000000BC000000200000009A000000B2
:10957400F4000000360000001D000000A9000000F7
:10958400E300000091000000610000005E000000A4
:10959400E60000001B000000080000006500000059
:1095A40099000000850000005F0000001400000026
:1095B400A000000068000000400000008D000000D2
:1095C400FF000000D8000000800000004D000000F3
:1095D40073000000270000003100000006000000B6
:1095E400060000001500000056000000CA0000003C
:1095F40073000000A8000000C90000006000000023
:10960400E20000007B000000C00000008C000000AD
:109614006B0000000000C93F0000F0390000DA3799
:109624000000A2330000842E0000502B0000C2274B
:109634000000D0220000C41F0000C61B0000441715
:0C96440004000000070000000900000006
:08965000CD840008FD010008B3
:04965800D90100082C
:10965C00FFFFFFFF0024F4000100000010000000D9
:10966C009D7300085573000861720008000000002B
:10967C0065710008F7710008CD710008000000004A
:10968C000000000000000000A97100089D71000896
:10969C00B5710008C171000809024300020100C045
:1096AC00320904000001020201000524001001052A
:1096BC00240100010424020205240600010705828E
:1096CC000308001009040100020A0000000705014C
:1096DC00024000000705810240000000090243001F
:1096EC00020100C03209040000010202010005243D
:1096FC0000100105240100010424020205240600C7
:10970C00010705820308001009040100020A000089
:10971C00000705010200020007058102000200009B
:10972C000A06000200000040010000000907430087
:10973C00020104C0320904000001020201000524E8
:10974C000010010524010001042402020524060076
:10975C00010705820308001009040100020A000039
:10976C0000070501024000000705810240000000CF
:10977C00897F0008617F0008657F00086D7F000805
:10978C00697F0008DD7F0008E97F0008AD800008D4
:10979C008980000875800008C9800008ED800008E9
:1097AC000000000012010002020200408304405736
:1097BC000002010203010000040309041A03000063
:1097CC00000000000000000000000000000000008D
:1097DC0000000000000000000000000074040020E5
:1097EC00DC04002044050020000000000000000004
:1097FC00000000000000000000000000000000005D
:10980C00000000000000000000000000000000004C
:10981C00000000000000000000000000000000003C
:10982C00000000000000000000000000000000002C
:10983C00000000000000000000000000000000001C
:10984C00000000000000000000000000000000000C
:10985C0000000000000000000000000000000000FC
:10986C0000000000000000000000000000000000EC
:10987C0000000000000000000000000000000000DC
:10988C0001000000000000000E33CDAB34126DE679
:10989C00ECDE05000B0000000000000000000000E2
:1098AC0000000000000000000000000000000000AC
:1098BC00000000000000000000000000000000009C
:1098CC00000000000000000000000000000000008C
:1098DC00000000000000000000000000000000007C
:049C0C00D020002044
:040000050800199D39
:00000001FF
